:020000040800F2
:10000000C4230020A1010008E9010008E90100085B
:10001000E9010008E9010008E9010008000000000A
:10002000000000000000000000000000E9010008DE
:10003000E901000800000000E9010008A9480008E3
:10004000E9010008E9010008E9010008E9010008E8
:10005000E9010008E9010008E9010008E9010008D8
:10006000E9010008D9370008E9010008E9010008A2
:10007000E9010008E9010008E9010008E9010008B8
:10008000E9010008E9010008E9010008E9010008A8
:10009000E9010008DD270008E9010008F937000838
:1000A000E901000879460008E9010008E9010008B3
:1000B000653C0008E901000800000000E9010008B3
:1000C000E90100080000000000000000E90100084C
:1000D0000000000081360008E9010008000000006F
:1000E000C5270008E9010008E90100080000000038
:1000F0000000000000000000000000000000000000
:1001000000000000000000005FF808F10348044B05
:10011000834202D0034B03B1184770478C03002081
:100120008C030020000000000548064B1B1AD90F65
:1001300001EBA301491002D0034B03B118477047EC
:100140008C0300208C0300200000000010B5064C3A
:10015000237843B9FFF7DAFF044B13B10448AFF338
:1001600000800123237010BD9003002000000000D8
:10017000C497000808B5054B1BB105490548AFF306
:100180000080BDE80840FFF7CFBF00BF00000000BF
:1001900094030020C4970008EFF31080704700001C
:1001A00008B50C4B0C4A03E052F8041B43F8041B3F
:1001B0000A498B42F8D30A480A494FF000028842A4
:1001C000B8BF40F8042BFADB00F078F804F0D4FA5A
:1001D00008BD00BF00000020CC9700088C03002061
:1001E00090030020C81F002008B504F0C5FA632260
:1001F0001146502002F0B0FB08BD000082B0002381
:1002000001932A4A136843F480331360274B1B6819
:1002100003F400330193019B002BF7D0234B1B68A1
:1002200013F4003F06D001230193019B012B04D05E
:1002300002B0704700230193F7E71D4B1A6842F0A4
:1002400010021A601A6822F003021A601A6842F05B
:1002500002021A60A3F580535A685A605A685A60BD
:100260005A6842F480625A605A6822F47C125A60DA
:100270005A6842F4E8125A601A6842F080721A60B2
:100280000A4B1B6813F0007FFAD0084B5A6822F023
:1002900003025A605A6842F002025A60034B5B68DC
:1002A00003F00C03082BF9D1C2E700BF0010024095
:1002B0000020024008B5FFF7A1FF08BD08B5104BAC
:1002C0001A6842F001021A6059680E4A0A405A60E0
:1002D0001A6822F0847222F480321A601A6822F4BA
:1002E00080221A605A6822F4FE025A604FF41F02FC
:1002F0009A60FFF7DFFF044B4FF000629A6008BD81
:10030000001002400000FFF800ED00E010B4426869
:1003100022F4702222F480720B6891F804C043EA40
:100320000C231343436083680A4A1A40CB688C68E5
:10033000234391F805C043EA4C0313438360C36A27
:1003400023F470030A7C013AD2B243EA0253C36237
:1003500010BC7047FDF7F1FF21B1836843F0010342
:1003600083607047836823F001038360704721B185
:10037000836843F4807383607047836823F48073D9
:1003800083607047836843F0080383607047836825
:1003900013F0080F01D001207047002070478368D8
:1003A00043F0040383607047836813F0040F01D0A7
:1003B000012070470020704721B1836843F4A003F7
:1003C00083607047836823F4A0038360704710B58F
:1003D00009291ED9C468A1F10A0C0CEB4C0C4FF092
:1003E000070E0EFA0CFE24EA0E0403FA0CFC44EA93
:1003F0000C04C460062A1BD8436B013A02EB82024C
:100400001F24944023EA040301FA02F213434363D6
:1004100010BD046901EB410E4FF0070C0CFA0EFC05
:1004200024EA0C0C03FA0EF34CEA03030361E1E740
:100430000C2A0CD8036B073A02EB82021F2494406B
:1004400023EA040301FA02F213430363E0E7C36AF9
:100450000D3A02EB82021F24944023EA04039140E8
:100460000B43C362D4E71AB143690B43436170473E
:10047000436923EA0103436170470000036823F0E6
:1004800001031B041B0C03600023036043608360B3
:10049000C360364B984221D0354B984224D0354B1F
:1004A000984227D0344B98422AD0344B98422DD0D2
:1004B000334B984230D0334B984233D0324B984232
:1004C00036D0324B984239D0314B98423CD0314BE8
:1004D00098423FD0304B984242D070472F4A5368E1
:1004E00043F00F03536070472C4A536843F0F00306
:1004F00053607047294A536843F4706353607047F0
:10050000264A536843F4704353607047234A536844
:1005100043F4702353607047204A536843F47003D8
:10052000536070471D4A536843F0706353607047CF
:100530001B4A536843F00F0353607047184A5368CF
:1005400043F0F00353607047154A536843F47063F7
:1005500053607047124A536843F4704353607047C6
:100560000F4A536843F470235360B6E70800024013
:100570001C0002403000024044000240580002408B
:100580006C00024080000240080402401C0402404B
:10059000300402404404024058040240000002407B
:1005A0000004024021B1036843F001030360704777
:1005B000036823F001031B041B0C03607047000059
:1005C000044B00221A605A609A60DA60024A5A614B
:1005D000704700BF00040140FFFF0F008379002B2C
:1005E00035D010B41F4B1A68016822EA01021A6064
:1005F0005A68016822EA01025A60027902F18042D7
:1006000002F5823211680468214311609A6801681A
:1006100022EA01029A60DA68016822EA0102DA60DD
:100620004379102B09D003F1804303F582331A6814
:1006300001680A431A6010BC70470A4B9A68016847
:100640000A439A60DA6801680A43DA60F3E70379DB
:1006500003F1804303F582331A68016822EA01023C
:100660001A60704700040140064A1368034052694B
:10067000024202D01BB900207047002070470120C1
:10068000704700BF00040140014B5861704700BF34
:1006900000040140034B044A5A6002F188325A6058
:1006A000704700BF0020024023016745024A1369DA
:1006B00043F080031361704700200240104BDB6859
:1006C00013F0010F17D10E4BDB6813F0040F0BD1A1
:1006D0000B4BDB6813F0100F0FD0094AD36843F0BF
:1006E0001003D36003207047054AD36843F0040326
:1006F000D36002207047012070470420704700BF7C
:100700000020024010B50446FFF7D8FF02E0FFF7D3
:10071000D5FF013C012801D1002CF8D104B110BD56
:100720000520FCE738B504464FF43020FFF7EAFF18
:10073000042800D038BD0A4D2B6943F002032B6119
:100740006C612B6943F040032B614FF43020FFF7BD
:10075000D9FF2B6923F00203DB04DB0C2B61E9E7F3
:100760000020024030B583B005460C4600230193BB
:100770004FF40050FFF7C6FF042801D003B030BD8E
:10078000124A136943F001031361A3B22B804FF4A3
:100790000050FFF7B7FF042807D00C4A136923F075
:1007A0000103DB04DB0C1361E8E702350195019BD3
:1007B000210C19804FF40050FFF7A4FF034A13697E
:1007C00023F00103DB04DB0C1361D7E700200240B8
:1007D00030B5CB7803F00F02964613F0100F03D01C
:1007E00091F802E04EEA020E0B78FBB10568002397
:1007F00001E042610133072B17D801229A40B1F87A
:1008000000C032EA0C0CF5D19C004FF00F0C0CFA32
:1008100004FC25EA0C050EFA04F42543CC78282CB8
:10082000E7D0482CE6D10261E4E705600B88FF2B96
:1008300025D94568002303E0CC78482C1CD001332F
:10084000072B1BD803F1080C012202FA0CF2B1F8B5
:1008500000C032EA0C0CF2D19C004FF00F0C0CFAE5
:1008600004FC25EA0C0C0EFA04F444EA0C05CC78DE
:10087000282CE1D14261DFE70261E0E7456030BD4D
:10088000016170474161704710B401F003029200AA
:100890004FF00F0C0CFA02FC8908084B023153F898
:1008A000214024EA0C0443F8214053F821409040B1
:1008B000044343F8214010BC704700BF00000140D2
:1008C000024B4AF6AA221A60704700BF003000406F
:1008D00040F0BF6040F40030014BD860704700BF6B
:1008E00000ED00E01B4BDA68D243C2F30222042A77
:1008F00000D90422C2F10401C9B20F231341427886
:100900008A40D2B281780B4013431B01DBB20278DC
:1009100002F1604202F5614282F80033C378012B94
:100920000CD0017890F9003001F01F015B09012221
:100930008A402033084941F823207047017890F914
:10094000003001F01F015B0901228A40024941F891
:100950002320704700ED00E000E100E021F060415D
:1009600021F07F010143014B9960704700ED00E0E9
:10097000034A536823F4404303435360704700BF66
:100980000010024010B4294B5B6803F00C03042BE9
:100990002BD0082B2CD013B1254B036001E0244B46
:1009A000036022494B68C3F30313224CE25CD2B2CA
:1009B0000368D34043604A68C2F30222A25CD2B209
:1009C00023FA02F282604A68C2F3C222A25CD2B267
:1009D000D340C3604A68C2F3813217498A5CD2B2FD
:1009E000B3FBF2F3036110BC7047114B0360D8E70F
:1009F0000E4A53685268C3F38343023312F4803FB4
:100A000004D10E4A02FB03F30360CAE7074A5268A7
:100A100012F4003F04D0094A02FB03F30360C0E76D
:100A2000034A02FB03F30360BBE700BF0010024070
:100A300000127A00080000200400002000093D0098
:100A400021B1054A5369034353617047024A536910
:100A500023EA0003536170470010024021B1054AA8
:100A60009369034393617047024A936923EA000341
:100A7000936170470010024021B1054AD3690343D6
:100A8000D3617047024AD36923EA0003D3617047F8
:100A9000001002402DE9F041028802F441520F8813
:100AA000B1F802808E88CD880C89B1F80AE0B1F8DF
:100AB0000CC0CB8947EA08073E4335432C434EEA36
:100AC000040E4CEA0E0C43EA0C0313430380838BA1
:100AD0009BB223F400639BB283830B8A0382BDE83D
:100AE000F08129B103889BB243F040030380704733
:100AF00003889BB223F040039BB20380704781813F
:100B000070470389194201D00120704700207047C7
:100B100003889BB2104A904206D0B0F1804F03D0B8
:100B2000A2F59432904203D123F070034A88134314
:100B300023F440739BB2CA88134303808B88838558
:100B40000B880385044B984202D0012383827047AF
:100B50000B7A0386F9E700BF002C014010B5038C27
:100B60009BB223F001039BB20384028C92B2B0F8D3
:100B700004E01FFA8EFE038B9BB223F073030C88F4
:100B8000234322F002020C892243B1F802C04CEA4E
:100B900002020D4CA04206D0A0F804E00383CB88EB
:100BA0008386028410BD22F008024C89224322F081
:100BB00004028C8822432EF4407E8C894EEA040E77
:100BC000CC8944EA0E0EE7E7002C014000B5038C07
:100BD0009BB223F010039BB20384028C92B2B0F854
:100BE00004E01FFA8EFEB0F818C01FFA8CFC2CF43B
:100BF000E64C0B881B029BB24CEA030C22F020024D
:100C00000B891B019BB21A434B881B019BB21343F8
:100C1000124A904208D0A0F804E0A0F818C0CA8890
:100C2000028703845DF804FB23F080034A891201E4
:100C300092B2134323F040038A88120192B2134305
:100C40002EF4406E8A89920092B24EEA020ECA8950
:100C5000920092B242EA0E0EDDE700BF002C014086
:100C600000B5038C9BB223F480739BB20384028C87
:100C700092B2B0F804E01FFA8EFEB0F81CC01FFA62
:100C80008CFC2CF0730C0B884CEA030C22F40072E1
:100C90000B891B029BB21A434B881B029BB2134366
:100CA000134A904203D002F50062904217D123F418
:100CB00000634A89120292B2134323F480638A8844
:100CC000120292B213432EF4405E8A89120192B24C
:100CD0004EEA020ECA89120192B242EA0E0EA0F842
:100CE00004E0A0F81CC0CA88828703845DF804FB76
:100CF000002C0140704770B50D884E888C88B1F883
:100D000006E0B1F808C04A898B8945EA060121430B
:100D10004EEA01014CEA01010A431343A0F84430B2
:100D200070BD4FF6FF73838000230380C380438030
:100D3000037270470023038043808380C380038154
:100D400043818381C3817047002303804380838074
:100D5000C380038143818381704729B103889BB29B
:100D600043F001030380704703889BB223F0010323
:100D70009BB20380704729B103889BB243F0800384
:100D80000380704703889BB223F080039BB20380EB
:100D9000704729B183889BB243F008038380704772
:100DA00083889BB223F008039BB283807047038B38
:100DB0009BB223F008030B4303837047038B9BB262
:100DC00023F40063090289B20B4303837047838BCA
:100DD0009BB223F008030B4383837047838B9BB242
:100DE00023F40063090289B20B438383704729B15E
:100DF00003889BB243F004030380704703889BB2CF
:100E000023F004039BB203807047028A83890B405E
:100E1000114202D01BB9002070470020704701200A
:100E20007047C94389B201827047000030B587B06E
:100E300004460D46038A9BB2CA8823F440531343E9
:100E4000038283899BB2898828896A8901430A437E
:100E500023F4B05323F00C031343A381A38A9BB262
:100E6000AA8923F440731343A38201A8FFF78AFDE4
:100E70001D4B9C4224D0039BA28912F4004F21D128
:100E800003EB830303EB83032A689200B3FBF2F3C3
:100E9000164AA2FB031252091101642002FB10330F
:100EA000A28912F4004F16D11B0132330F4AA2FB64
:100EB0000323C3F343130B439BB2238107B030BD1D
:100EC000049BD9E703EB830303EB83032A685200F7
:100ED000B3FBF2F3DCE7DB003233044AA2FB03236B
:100EE000C3F342130B43E7E7003801401F85EB5182
:100EF00029B183899BB243F400538381704783896E
:100F00009BB223F400539BB283817047C1F3421C10
:100F100001F01F0101238B40BCF1010F08D0BCF18F
:100F2000020F07D014303AB10268134303607047D0
:100F30000C30F8E71030F6E7026822EA030303609A
:100F400070470388194201D0012070470020704784
:100F500084460023184600E001338B4206D25CF839
:100F60002320B2F1FF3FF7D01044F5E770470000AF
:100F700010B54FF0010C0CFA01FCD0F8004244F01F
:100F80000104C0F80042D0F81C4224EA0C04C0F866
:100F90001C42D0F80C4244EA0C04C0F80C42D0F8D1
:100FA000044224EA0C04C0F80442CBB1D0F8143255
:100FB00043EA0C03C0F814324831174B40F8313083
:100FC00000EBC10103F1C0434B609DF80830012BD9
:100FD0001BD0D0F8003223F00103C0F8003210BD5E
:100FE0006FEA0C0ED0F814320EEA0303C0F8143284
:100FF000D20442F0004242F00402483140F831206D
:1010000000EBC101054B4B60DFE7D0F81C3243EA2F
:101010000C03C0F81C32DCE7040004800400FCE789
:1010200070B582B006460D460024072C11D815F87D
:1010300004C0BCF1FF0F02D00134E4B2F5E7211D7A
:101040000123009300233246C9B20848FFF790FFFE
:101050002E55082C01D002B070BD33460E22C1219E
:101060004FF4006001F013FCF5E700BF006400409E
:1010700030B583B00D460024072C0FD82B5D83427A
:1010800002D00134E4B2F7E7211D00230093FF22D0
:10109000C9B20348FFF76CFFFF232B5503B030BDE7
:1010A000006400400023032B08D80D4A1A4492F82C
:1010B000C821824210D00133DBB2F4E70023072BB2
:1010C00008D8074A1A4492F8CC21824206D001334C
:1010D000DBB2F4E700207047012070470120704721
:1010E0002004002023281BD8232817D8DFE800F08D
:1010F0001416162C12161616161616161616161680
:101100001614142C16161216161616161616161671
:1011100014161630042070470120704708207047CD
:101120004B2817D830280BD33038C0B20123834066
:10113000094A13420AD113F0310F03D10820704736
:101140000820704704207047062070470020704731
:1011500002207047082070478800F00D30B585B038
:1011600004460568C5F3C62531212846FFF7BAFFB6
:10117000227902F00F02824202D1002005B030BD78
:10118000E378029201900095C3F3C1030A22C121C2
:101190004FF4806001F034FB0A20EFE703468268D9
:1011A00012F0806F09D1826812F0006F2AD1826834
:1011B00012F0805F28D0022000E0002000B500F18E
:1011C00018024FEA021C03EB0212D1F800E043F8C8
:1011D0000CE0D1F804E0C2F804E003EB0012D1F80F
:1011E00008E0C2F888E1C968C2F88C1153F80C20F5
:1011F00042F0010243F80C20044B0822A3F8BE2160
:101200005DF804FB0120D9E704207047200400208A
:1012100008B501460148FFF7C1FF08BD0064004062
:10122000094AB2F82432013BA2F82432B2F8223241
:1012300001339BB2A2F82232802B00D070471346B4
:101240000022A3F82222F9E72014002030B51E4B1B
:10125000C31A18BF012384684FEAC10C802202FA26
:101260000CF214422FD184684FF0080E0EFA0CFCD9
:1012700014EA0C0F1DD003EB43040C447434134DDB
:1012800005EB840CDCF804400134CCF80440042C59
:1012900019D984682243826003EB43030B44002086
:1012A000CCF80400783355F82310013145F82310A9
:1012B00009E003EB4303194401F17403034A02EB11
:1012C000830300225A6030BD0064004020040020E7
:1012D00038B51C4B9B6803F0083323F00063FBB95F
:1012E0000024022C26D8184B5B6A13F4801F23D0ED
:1012F000164BB3F824320BB3134D05F58053B3F8F6
:101300002202A23005EB0010FFF782FF0523A5F8AB
:10131000BE31042814D0FFF783FF0134E4B2E0E7C4
:101320000024022CDCD821460648FFF78FFF013449
:10133000E4B2F6E7002038BD0020FCE70020FAE721
:101340000620F8E70064004020040020201400205C
:1013500008B50C4BB3F824327F2B08D80A4800F5A7
:101360008053B3F82032A23300EB031008BDFFF71F
:1013700057FF80230C22C1214FF4805001F087FADF
:101380000020F3E7201400202004002010B50446BC
:10139000C378042262F34713C370037813430370C6
:1013A000C37813F0180F0CBF01220022037862F3F8
:1013B00041030370DBB26FF3000303700068C0F3F6
:1013C000C620FFF78FFE237960F30303237110BD5E
:1013D00010B504463121FFF7D9FF184B5B6A13F4AF
:1013E000801F03D0164BB3F82432CBB1FFF7B0FF08
:1013F000844600B3844203D094E80F008CE80F00C9
:101400000F4AB2F824320133A2F82432B2F8203263
:1014100001339BB2A2F82032802B08D0002010BDEF
:101420002046FFF7F5FE0428E0D00020F7E7002073
:10143000A2F82002F3E70C20F1E700BF200400200F
:1014400020140020F8B507460E4615461C46FFF747
:101450007FFFE8B1C37867F3C403C370438866F3C2
:10146000CA034380036865F3D123036083789DF842
:10147000182062F382038370038864F3CA03038035
:10148000079BD3E90023C0E90223FFF7A1FFF8BDC2
:101490000C20FCE7F8B507460E4615461C46FFF73C
:1014A00057FFE0B1C378012262F3C403C3700D4B50
:1014B00093F82220438862F3CA034380036867F3EA
:1014C000D123036083786FF382038370038866F30C
:1014D000CA0303808560C460FFF77AFFF8BD0C2063
:1014E000FCE700BF2004002008B50A46002301469F
:1014F0004020FFF7CFFF08BD03680B6043684B60D7
:1015000083688B60C368CB607047C06810F00300CD
:1015100018BF01207047006910F0030018BF0120B8
:10152000704738B504460D46FFF7EFFF50B1294626
:1015300004F5D870FFF7E0FFE36843F02003E360B1
:10154000002038BD0220FCE738B504460D46FFF701
:10155000E2FF50B1294604F5E070FFF7CDFF2369A3
:1015600043F020032361002038BD0220FCE7000087
:1015700010B51848FFF7CFFF012806D00220164B00
:1015800093F80032012B20D010BD144BB3F8C200E9
:10159000C0F3C700FFF786FD18B10F4B93F8003278
:1015A00033B10C4A136943F0200313610220E6E7CC
:1015B0000B4C21460748FFF7C7FF22796FF304124F
:1015C0002271012222740020D9E7034B0822A3F8DC
:1015D000BC21D9E7006400402004002000650040E1
:1015E0001006002010B51F4BB3F81C3A7F2B07D80C
:1015F0001D48FFF78AFF01280BD00220C0B210BDA2
:1016000080230B22C1214FF4005001F040F90B2040
:10161000F5E7144CB4F8181A090101F506712144D4
:101620001148FFF77EFFB4F8183A04EB031292F862
:101630001C126FF3041182F81C12B4F81C2A013238
:10164000A4F81C2A01339BB2A4F8183A802B05D0C9
:10165000044B0822A3F8BC210020CFE70022A4F805
:10166000182AF5E7200400200064004038B51D4B1F
:1016700093F80032012B1FD01A4BB3F81C4A64B305
:101680001D46B3F81ACA03EB0C1303F5067305F5F0
:10169000027E0FCB8EE80F00013CA5F81C4A0CF12E
:1016A000010C1FFA8CFCA5F81ACABCF1800F0ED1F0
:1016B0000022A5F81A2A0AE00A4D05F5027405F57C
:1016C000F8730FCB84E80F00002385F8003206483A
:1016D000FFF744FD18B9012038BD0020FCE70020C9
:1016E000FAE700BF20040020280600202DE9F04181
:1016F00084B080460E46084607F0BCF8451C15E04D
:101700000821284600F0FCF8044602AF02463146A4
:10171000384607F0A1F8019700230093E3B24C226A
:1017200041460120FFF78EFE2D1B2644002DE7D1F8
:1017300004B0BDE8F08108B5FFF7CAFD08BD0000A0
:10174000B0F1FF3F09D0C0F30310012807D00228F1
:1017500007D040B1054B1868704700207047044817
:101760007047044870470448704700BF18000020C5
:10177000000C01400010014000080140B0F1FF3FA3
:1017800006D010B50446FFF7DBFF240C446110BD02
:101790007047B0F1FF3F06D010B50446FFF7D0FF09
:1017A000240C046110BD7047B0F1FF3F07D008B5AD
:1017B00011B9FFF7E3FF08BDFFF7EBFFFBE7704749
:1017C000B0F1FF3F31D010B50446FFF7B9FF04F088
:1017D0000F03072B11D89B0002680F21994022EAC2
:1017E000010202600268C4F3032101FA03F3134308
:1017F000036014F4004F12D110BD04F00F03083B36
:101800009B0042680F21994022EA0102426042682F
:10181000C4F3032101FA03F313434360E9E7C4F37C
:1018200000312046FFF7C0FFE6E77047B0F1FF3F09
:101830000AD010B50446FFF783FF806804F00F0458
:10184000E04000F0010010BD00207047B0F1FF3F04
:101850000AD010B50446FFF773FFC06804F00F0408
:10186000E04000F0010010BD0020704708B50A46B6
:10187000002106F0E7FF08BD074BDA6922EA000203
:10188000DA611A6902431A61DA690243DA611A6994
:1018900022EA00021A61704700100240074B9A6961
:1018A00022EA00029A61DA680243DA609A69024326
:1018B0009A61DA6822EA0002DA607047001002409A
:1018C00000B583B08DF804008DF8051000238DF865
:1018D000063001238DF8073001A8FFF703F803B0A5
:1018E0005DF804FB034608468B4200DD184670474E
:1018F000884203DD904202DB10467047084670477D
:10190000034608468B4200D21846704703460846F5
:101910008B4200D918467047884203D9904202D3BF
:10192000104670470846704770B582B005460C46B1
:10193000124E31608B7D00934B894A68497D207D32
:1019400000F0BFFA33689A7D012A01D902B070BD58
:1019500005EBC5056D000E359B8900932B461422BF
:101960002946002000F09BFA3368597D187D9B8939
:1019700000932B46802200F092FAE7E7C80300208C
:1019800030B583B00E4C21608B7D00934B894A6843
:10199000497D052000F095FA23681B68094D1A68F7
:1019A0000949284606F02EFF22689389517D107D53
:1019B000927D00922A4600F084FA03B030BD00BF49
:1019C000C8030020CC0300205091000830B583B03C
:1019D0000E4C21608B7D00934B894A68497D052020
:1019E00000F06FFA23681B68094D1A8809492846D8
:1019F00006F008FF22689389517D107D927D009248
:101A00002A4600F05EFA03B030BD00BFC8030020D4
:101A1000CC0300205491000830B583B00E4C2160F7
:101A20008B7D00934B894A68497D052000F049FA77
:101A300023681B68094D1A780949284606F0E2FE1A
:101A400022689389517D107D927D00922A4600F094
:101A500038FA03B030BD00BFC8030020CC0300201B
:101A60005C91000830B583B00E4C21608B7D0093F3
:101A70004B894A68497D052000F023FA23681B68DA
:101A8000094D1A880949284606F0BCFE2268938948
:101A9000517D107D927D00922A4600F012FA03B02B
:101AA00030BD00BFC8030020CC03002064910008B3
:101AB00030B583B00E4C21608B7D00934B894A6812
:101AC000497D052000F0FDF923681B68094D1A685F
:101AD0000949284606F096FE22689389517D107DBB
:101AE000927D00922A4600F0ECF903B030BD00BFB1
:101AF000C8030020CC0300206C91000830B583B0EF
:101B00000D4C21608B7D00934B894A68497D0520EF
:101B100000F0D7F92368094D1A680949284606F0EC
:101B200071FE22689389517D107D927D00922A4634
:101B300000F0C7F903B030BDC8030020CC0300207B
:101B40007491000830B583B0184C21608B7D0093F0
:101B50004B894A68497D052000F0B3F923681B686A
:101B60001D68284606F008FE044606F0EBFB014619
:101B7000284606F031FB0E4906F038FC06F0FCFD65
:101B8000031E11DB0B4D22460B49284606F03AFE98
:101B9000064B1A689389517D107D927D00922A46EA
:101BA00000F08FF903B030BD5B42EBE7C8030020C3
:101BB00000007A44CC030020789100080000000067
:101BC000F0B583B00C46284B19600B681888642860
:101BD00000D9642006F0BAF921A3D3E9002305F067
:101BE00039FF06F0A5FA0546A37D00936389626874
:101BF000617D052000F065F91B4B1F683E7DC6F135
:101C0000800006F09FFB294606F0F0FB04463046B4
:101C100006F098FB214606F0E1FA06F0D3FD84B207
:101C2000A64203D37F2C0DD903B0F0BD797DBB7DD7
:101C300003EBC3037A8900920B442246304600F03E
:101C400037F9EFE7084B1A68517D937D03EBC30327
:101C5000928900920B448022204600F029F9E3E7A4
:101C60007B14AE47E17A843FC803002030B583B0CF
:101C70000C460B4B19600B680A4DAC461868596846
:101C80009A68DB68ACE80F0000232B74A37D0093F7
:101C900063892A46617D052000F013F903B030BD49
:101CA000C8030020CC030020F0B583B00646234BC8
:101CB0001960234B00221A605A609A60DA601A6138
:101CC0000A6812681A60D3B21F2B02D81C4B2D2051
:101CD0001870C2F307231F2B02D8194B2D20587000
:101CE000C2F307431F2B02D8154B2D209870B2F179
:101CF000005F02D2124B2D22DA70114D20232B717E
:101D00000F680024053507E03A5D0E49284606F0C5
:101D100079FD03350134E4B2032CF5D9074B1A6879
:101D2000538906EBC60149000531927D0092044AB1
:101D3000C9B2052000F0C5F803B0F0BDC80300200B
:101D4000CC0300208091000830B583B0134D29608A
:101D500000EBC00044000534E4B28B7D00934B8956
:101D60004A682146052000F0ACF82B681B681B78F8
:101D70008BB90B4A0B4D0C49284606F043FD074B27
:101D80001A689389927D00922A462146592000F0D4
:101D900098F803B030BD054AECE700BFC803002047
:101DA00088910008CC0300207491000890910008ED
:101DB00038B50546002404E0E0B2FFF7B5FD013474
:101DC000A4B204EB440305EBC30155F83330002BF8
:101DD00054D00B7A0E2BF2D801A252F823F000BF98
:101DE000B91D00081D1E0008251E00082D1E000834
:101DF000351E00083D1E0008451E00084D1E000847
:101E0000551E0008BF1D00085D1E0008BF1D00080C
:101E1000651E00086D1E0008751E0008E0B2FFF781
:101E2000AFFDCCE7E0B2FFF7D1FDC8E7E0B2FFF7C6
:101E300089FEC4E7E0B2FFF7EFFDC0E7E0B2FFF7CD
:101E400011FEBCE7E0B2FFF733FEB8E7E0B2FFF700
:101E500055FEB4E7E0B2FFF777FFB0E7E0B2FFF777
:101E6000AFFEACE7E0B2FFF71FFFA8E7E0B2FFF775
:101E7000FDFEA4E7E0B2FFF717FFA0E738BD00BF03
:101E800038B504460D4600F0BBF82B46224600212B
:101E9000084600F0A5F9002000F0DAF938BD10B5C9
:101EA00082B0BDF81040009400F08EFA02B010BD70
:101EB00010B582B0BDF81040009400F035FB02B0C0
:101EC00010BD08B59DF808C0BCF1010F02D000F0AC
:101ED00045FC08BD00F01CFCFBE7000010B5044603
:101EE00002210848FEF70DFE0028F9D021460548DA
:101EF000FEF705FE80210348FEF703FE0128F9D016
:101F000010BD00BF0038004010B504464FF48041BA
:101F10000648FEF7B7FC2046FFF7E0FF80210448A3
:101F2000FEF7EFFD0128F9D010BD00BF000C014005
:101F30000038004010B504464FF480410648FEF7D3
:101F40009FFC2046FFF7CAFF80210448FEF7D9FD19
:101F50000128F9D010BD00BF000C0140003800403E
:101F600010B504464FF480512048FEF78BFC362014
:101F7000FFF7CAFF022C20D0032C2AD0012C0BD053
:101F80001B4B1A881B4B1A801B4B1A881B4B1A8041
:101F90000020FFF7CFFF0AE0174B1A88154B1A8075
:101FA000134B1A88154B1A80A020FFF7C3FF4FF47C
:101FB00080510E48FEF764FC10BD0F4B1A880D4B84
:101FC0001A800B4B1A880D4B1A806020FFF7B2FF66
:101FD000EDE7074B1A88074B1A80074B1A88074B07
:101FE0001A80C020FFF7A6FFE1E700BF000C014008
:101FF000FA030020F6030020F8030020F403002079
:102000002DE9F04186B006460D4601214FF480408F
:10201000FEF732FD01210820FEF720FD4FF420439A
:10202000ADF814304FF018088DF8178003278DF89D
:102030001670674C05A92046FEF7CAFB4FF4A4436F
:10204000ADF8143010238DF817308DF8167005A9EF
:102050002046FEF7BDFB01210820FEF7FFFC012111
:102060004FF48040FEF708FD05365A4B1E800535BB
:10207000594B1D804FF48273ADF80230ADF80C80DF
:102080004FF44043ADF800300025ADF80650ADF8F0
:1020900008500723ADF81030ADF80450ADF80E50DD
:1020A0004FF40076ADF80A60DFF8308169464046AB
:1020B000FEF7F0FC01214046FEF713FD4FF480517E
:1020C0002046FEF7DDFB31462046FEF7D9FB052012
:1020D00005F0BAFC31462046FEF7D4FB052005F09A
:1020E000B3FC31462046FEF7CBFB4FF4805120462F
:1020F000FEF7C6FB052005F0A7FC4FF480512046F3
:10210000FEF7C0FB1120FFF7FFFEB120FFF7FCFE3A
:102110004FF480412046FEF7B3FB0520FFF7DEFEBB
:102120003C20FFF7DBFE3C20FFF7D8FEB220FFF794
:10213000EBFE4FF480412046FEF7A2FB0520FFF79F
:10214000CDFE3C20FFF7CAFE3C20FFF7C7FEB320C0
:10215000FFF7DAFE4FF480412046FEF791FB0520A1
:10216000FFF7BCFE3C20FFF7B9FE3C20FFF7B6FEB0
:102170000520FFF7B3FE3C20FFF7B0FE3C20FFF741
:10218000ADFEB420FFF7C0FE3846FFF7D3FE3A207D
:10219000FFF7BAFE0520FFF7CDFE2020FFF7B4FEC3
:1021A0001320FFF7B1FE2620FFF7AEFE0120FFF758
:1021B000C1FE2920FFF7A8FE4FF480512046FEF70C
:1021C0005FFB2846FFF7CCFE06B0BDE8F08100BFFC
:1021D000000C0140FA030020F80300200038004002
:1021E0002DE9F04107460D4616461C462A20FFF70A
:1021F0008BFEDFF858804FF480414046FEF740FBED
:10220000380AFFF76BFEF8B2FFF768FE300AFFF7F7
:1022100065FEF0B2FFF762FE2B20FFF775FE4FF46C
:1022200080414046FEF72CFB280AFFF757FEE8B234
:10223000FFF754FE200AFFF751FEE0B2FFF74EFE13
:102240002C20FFF761FEBDE8F08100BF000C0140CB
:1022500070B5060AC5B2174C4FF480512046FEF700
:1022600011FB154B1B88013B144A1288013A9BB2A3
:1022700092B200210846FFF7B3FF4FF48041204699
:10228000FEF7FEFA002407E03046FFF727FE284657
:10229000FFF724FE0134A4B2084B1B88064A1288BB
:1022A00002FB03F39C42EFDB4FF480510148FEF741
:1022B000E7FA70BD000C0140F4030020F603002093
:1022C000F8B505460E4614460E4F4FF48051384679
:1022D000FEF7D8FA33462A4631462846FFF780FFF4
:1022E0004FF480413846FEF7CBFA200AFFF7F6FD9F
:1022F000E0B2FFF7F3FD4FF480513846FEF7C0FA25
:10230000F8BD00BF000C01402DE9F84306460F461A
:1023100014464FEA1328DDB2DFF848904FF480519D
:102320004846FEF7AFFA23463A4621463046FFF7C5
:1023300057FF4FF480414846FEF7A2FA002407E019
:102340004046FFF7CBFD2846FFF7C8FD0134A4B295
:10235000BB1B9C42F4DD4FF480510248FEF790FA1B
:10236000BDE8F883000C01402DE9F84304460E4611
:1023700017464FEA1328DDB2DFF848904FF480513A
:102380004846FEF77FFA3B46224631462046FFF795
:1023900027FF4FF480414846FEF772FA002407E019
:1023A0004046FFF79BFD2846FFF798FD0134A4B295
:1023B000B81B8442F4DD4FF480510248FEF760FA06
:1023C000BDE8F883000C01402DE9F04F83B086464C
:1023D0008C4692469B46BDF8307095B280B22B1A5F
:1023E0001FFA83F91BB21FFA8BF689B2721A94B2E4
:1023F000009412B2002B24DD4FF00108002A23DDE7
:10240000012423B382B31FFA88F808FB09F91FFAE5
:1024100089F30FFA89F21FFA84F9009909FB01F494
:10242000A6B224B25100009161000191A24253DB97
:102430008CB2A4EB030B0FFA8BFBCDF8049066462D
:102440002AE04FF0FF38D9E74FF0FF34D9E7E345F2
:1024500004DD3B463246FFF787FF3AE03B460A463B
:102460003146FFF781FF34E0F24505DD3B460A4681
:102470002946FFF749FF2CE03B460A46014628461D
:10248000FFF742FF25E0009BE31A9BB25B440FFA83
:1024900083FB019B4B441EB2D64512D01FFA8EF52A
:1024A0001FFA86F93A4649462846FFF709FF454490
:1024B0000FFA85FEBBF1000FE5DAA3440FFA8BFBA0
:1024C000EAE7B4463A461FFA8CF11FFA8EF0FFF79E
:1024D000F7FE03B0BDE8F08FBDF800A0AAEB06063A
:1024E00036B2CDF80080754608E0019BAAEB0303E5
:1024F0009BB233441EB2009B43441DB2DC4510D056
:102500001FFA85F81FFA8CF43A4621464046FFF739
:10251000D7FE4C440FFA84FC002EE6DA564436B25D
:10252000ECE7AE46CEE700002DE9F84F04468846BA
:1025300091469A46BDF82860131AAAEB01050135A9
:1025400003FB0555ADB2370AF6B2DFF848B04FF4D9
:1025500080515846FEF796F953464A464146204672
:10256000FFF73EFE4FF480415846FEF789F90024FC
:1025700007E03846FFF7B2FC3046FFF7AFFC013406
:10258000A4B2AC42F5D34FF480510248FEF778F97B
:10259000BDE8F88F000C01402DE9F04182B00446FF
:1025A0000D461F0ADEB2A2F1200303EB8303224A89
:1025B0009918D05800900B798DF80430DFF87C80A2
:1025C0004FF480514046FEF75DF9AB1D221D9BB2D2
:1025D00092B229462046FFF703FE4FF48041404661
:1025E000FEF74EF900251BE00020FFF777FC0020E6
:1025F000FFF774FC0134A4B2042C0FD804F10803D3
:102600006B4413F8083C2B4113F0010FECD0384613
:10261000FFF764FC3046FFF761FCEBE70135ADB234
:10262000062D01D80024E7E74FF480510348FEF758
:1026300027F902B0BDE8F08164920008000C014067
:102640002DE9F04F83B001900E469A46A2F1200B7F
:102650005FFA8BFB0BEB8B0B2C4B9B444FF0000971
:1026600049E0002231462046FFF72AFE671CBFB230
:10267000002231463846FFF723FE06F101081FFA13
:1026800088F8002241462046FFF71AFE0022414604
:102690003846FFF715FE0234A4B20135EDB2042D21
:1026A00023D87F2C21D81BF8053043FA09F313F007
:1026B000010FD6D0524631462046FFF701FE671C77
:1026C000BFB2524631463846FFF7FAFD06F101081F
:1026D0001FFA88F8524641462046FFF7F1FD524660
:1026E00041463846FFF7ECFDD5E70236B6B209F1B0
:1026F00001095FFA89F9B9F1060F04D87F2E02D8D3
:10270000019C0025CBE703B0BDE8F08F6492000880
:10271000F8B504460E4615461F4607E00D4B1A88CD
:10272000083A964212DA0836F6B200242A7882B1C4
:1027300001353B4631462046FFF72EFF064B1888F1
:1027400006388442EADA0634E4B2EFE7002634467B
:10275000ECE7F8BDF4030020F6030020F8B50446CA
:102760000E4615461F4607E00D4B1A88103A964252
:1027700012DA1036F6B200242A7882B101353B46CF
:1027800031462046FFF75CFF064B18880C38844220
:10279000EADA0C34E4B2EFE700263446ECE7F8BDA1
:1027A000F4030020F60300200449CA6802F4E06242
:1027B000034B1343CB60BFF34F8FFEE700ED00E008
:1027C0000400FA0508B5044BDB6913F0040F00D1CF
:1027D00008BD02F08FFAFBE72004002008B5074B84
:1027E0005B6913F0100F04D0044B1B6913F0030F47
:1027F00000D108BDFEF7BCFEFBE700BF006400404F
:1028000038B50446002061F3070062F30F206FF330
:102810001F40002163F307019DF8103063F30F217F
:102820009DF8143063F317419DF8183063F31F616E
:102830000C4B9C4204D00C4BD3F8C431234202D140
:10284000094B5B6803B138BD074D0B460246297A38
:102850004220FEF71FFED5F8C4312343C5F8C4312A
:10286000F1E700BFEFBEADDE2004002010B584B05C
:10287000BDF818C04FEA1C2402945FFA8CF401944E
:102880001C0A0094DBB2FFF7BBFF04B010BD10B50B
:1028900084B01C0E0294C3F307440194C3F30724CD
:1028A0000094DBB2FFF7ACFF04B010BD00B585B0FB
:1028B0000023029301930093FFF7A2FF05B05DF898
:1028C00004FB30B585B093F803C01C68C4F3C6247C
:1028D0001D7905F00F0502951D88C5F3C705019503
:1028E0000094CCF3C103FFF78BFF05B030BD7047F8
:1028F00000B585B00A4B93F83B20029293F83A203A
:10290000019293F83920009293F838300122C421C3
:102910004FF48040FFF774FF05B05DF804FB00BF83
:10292000200400207047000008B5084BDB6813F056
:10293000807F00D108BD064BB3F8B417003918BF2B
:102940000121044B1868FEF72FFFF3E72004002055
:1029500020140020601E00207047000008B5054BC1
:102960005B681BB1013B034A536003B108BDFFF72D
:102970001BFF00BF200400203E4B4AF6AA221A602B
:102980003D4B5B6A13F0010F12D03C4BB3F8463657
:10299000002B6ED0013B9BB2384AA2F84636002B82
:1029A00067D1A2F580535A6A6FF300025A627047EA
:1029B00030B585B0304B93F82220FE2A47D05B6AB1
:1029C00013F4801F06D02C4B5B6A13F4001F24D035
:1029D00005B030BD01230093002319462848FEF7B7
:1029E000C7FA254B93F8220083F8C801002209E0BA
:1029F00002F1A201204B03EB0113598860F3CA01D5
:102A0000598001321D4BB3F824329342F0DC1A4A4C
:102A1000536A43F480135362D5E702AD294601207F
:102A200002F0D4FA144C019500230093402294F84C
:102A300022100120FEF706FD636A43F4001363626F
:102A4000052004F089FB0F4B01221A80C0E70A4BD6
:102A5000D3F8F830002BBBD093F82420012AB7D14B
:102A6000B3F91C20044B83F82220042004F074FBEB
:102A7000AEE7704700300040200400202014002002
:102A800000640040A81C002000207047024B002278
:102A900083F81021704700BF2004002010B50446C1
:102AA000406BB0F1FF3F08D10020237913F0080FED
:102AB00000D1C04300F0010010BDFEF7C7FEF4E7EF
:102AC0004911B0F9283003FB01F1B0F92E3091FB28
:102AD000F3F15211B0F92A3003FB021080B27047B3
:102AE00038B50446436C6BB1B3F90050A06905F0EA
:102AF00043FE01B2B4F92430AB4205DD0023A381CB
:102B0000E38138BD0F4DF1E7637913F0100F06D064
:102B10008D4202DA0023E381F3E76423FBE7A38D10
:102B2000CB1A9D4203DA0023A381E381E9E76A1A05
:102B300012B22046FFF7C4FF62890021FEF7ECFEC7
:102B4000E081DEE70180FFFF2DE9F041044687695F
:102B50004149384605F040FB404905F047FC404EEE
:102B600030604FF07E5105F039FB054630603D4A3C
:102B7000138801339BB21380052B02D91346002220
:102B80001A80A66C0021304605F0C4FD00282DD126
:102B9000B4F9260005F0D6FB0146304605F0E2FD0B
:102BA00020BB3146384605F017FB06462E4905F096
:102BB000BBFD00B32B4B1B889BB92C49304605F05D
:102BC000B3FD70B1E56C284605F0D2F920A3D3E936
:102BD000002305F0A3FA20B12549284605F0FCFAA8
:102BE000E0640023A381A389E38102E00023A381A1
:102BF000E381BDE8F0813146284605F0F7FB054644
:102C0000D4F84C804146384605F0F0FB0146284692
:102C100005F0E4FA05F0B0FDA081124B1B88002BF3
:102C2000E1D14FF07E51304605F09CFD0028DAD00E
:102C30004FF07E51404605F077FD0028D3D00C4977
:102C4000404605F0CBFAE064CDE700BFAFF300806B
:102C50007B14AE47E17AA43F0000C8420AD7233C68
:102C60002403002028030020CDCC4CBE0000A0C0CF
:102C70006F12833A08B5044BD3F8643703FB00F0B6
:102C8000800AFEF749FE08BD2014002010B5144646
:102C9000244B9A6942F004029A61DA6942F0010217
:102CA000DA612148FEF78CFD4FF080438C221A85B3
:102CB00040F2E7329A85B4F5807F2AD91B4BA3FBFB
:102CC0000423E41A03EB54031B0A03EB83035B00A6
:102CD0009BB24FF0804293874FF080431A8B92B2A1
:102CE00022F4E04292B21A831A8B92B242F4C042AA
:102CF0001A831A8B92B242F400621A831A8C92B22F
:102D000042F010021A841A8892B242F001021A802C
:102D100010BD04EB84046400A4B24FF080439C8790
:102D2000DAE700BF00100240029B040021F1D490BA
:102D300000B583B00123009300231A46FFF7A6FFD6
:102D400003B05DF804FB0000084B1B6913F4807F9F
:102D500000D0704710B50446FEF71BFD2046FEF775
:102D600018FD2046FEF70AFD10BD00BF200400201C
:102D700008B5074B5B6A13F0010F00D10020B0FAD1
:102D800080F14909034B1868FEF70EFD08BD00BF2E
:102D900020040020541E002008B5114BDB6813F0FE
:102DA000010F0CD10E4BDB6813F4803F06D00023DB
:102DB0004FF0804293870B4AC2F8503608BD00217D
:102DC0004FF08040FDF7C9FF064B0020A3F88C07A9
:102DD00083F8690783F86807FFF7CAFFE2E700BFD7
:102DE000200400202014002038B5234B1B783BB36F
:102DF0000546214BDB68002B23DB01F0010413F4B3
:102E0000003F03D01D4B5B68AB421CD06C862B7916
:102E100013F0080F01D184F00104184B5B68AB423A
:102E200016D0164B1B68AB421CD095F84030022BD5
:102E300006D0E86B0BB984F001042146FEF7B4FC20
:102E400038BD0021D9E7002CE0D1FFF7A5FFDDE771
:102E50001CB10B4B20221A61E3E7094B4FF400121F
:102E60001A61DEE71CB1074B01221A61DDE7054B51
:102E70004FF480321A61D8E7200400201C030020A0
:102E800000080140000C01408378023BDBB2022BBA
:102E90003ED810B50446038A01339BB203820289EF
:102EA00093422ED300230382438A01339BB2438291
:102EB0004289934207D300234382437913F0020FE0
:102EC00001D0C3898381A289A38A9A4200D9A381B0
:102ED000237913F0010F15D1A189638A994294BF18
:102EE00000210121237913F0020F07D0094B93F839
:102EF0006837013BDBB2012B00D900212046FFF7E8
:102F000073FF10BDA17C207B04F01EFC0146E9E7A5
:102F1000704700BF201400208378042B00D0704736
:102F200070B50446037903F03002302A09D013F05B
:102F3000200F34D113F0100F34D12046FFF7A6FD37
:102F400070BD1A4B5D688542F7D1194BD3F800313B
:102F5000B3F91C60A86905F00FFC28B9134B1A6877
:102F600000239381EB81E8E7864202DDB6F57A5FC4
:102F70000ADB0E4B1A68002191701868FFF734FFC6
:102F80002046FFF7E1FDD8E7084B1A680121917050
:102F90001868FFF729FF2046FFF7A2FDCDE7FFF7EE
:102FA0009FFDCAE7FFF7D0FDC7E700BF1C03002065
:102FB0002004002010B54FF080439B8F9BB2074A3E
:102FC000A2FB0323DB08064A1380064C2068FFF7A8
:102FD000A3FF6068FFF7A0FF10BD00BFCDCCCCCC35
:102FE0001C0400201C03002010B50446274BDB689E
:102FF00013F0007F15D0264BD3F808381A78022A30
:103000002BD0012814BF002101211869FEF7CCFB49
:10301000012C33D04FF0FF321D4BC3F81428C3F8F6
:103020003C281A4BDB6813F0007F15D1174B03F5D2
:10303000805282F844461B6913F4807F0CD1A2F5BC
:1030400080535B6A13F4007F1AD084F0010101F011
:1030500001011048FEF7A8FB10BD012814BF002194
:1030600001211869FEF7A0FB012C05D04FF0FF32BB
:10307000074BC3F86428D4E70122F9E70122CBE724
:1030800021460448FEF790FBE6E700BF200400203D
:103090002014002009C2000270B505460C46FDF759
:1030A0007BF8064672B6214B93F86837A34221D0CD
:1030B000012C28D00122934227D00120FFF758FE8F
:1030C000012C14BF00200120FFF78EFF174B0022B8
:1030D00083F8692783F86847ADB2A3F88C57012CB1
:1030E00021D0124BB3F888171148FFF721FE06B91B
:1030F00062B670BD0D4AB2F88C379BB22B449BB2BE
:10310000A2F88C37F3E70322D5E7084BB3F88C37E6
:103110009BB2AB4205D2054BB3F88C379BB2ED1A8C
:10312000CBE70125C9E7B3F88417DDE720140020B9
:10313000FC1A002008B50F4BDB6813F0010F09D013
:103140000D4BB3F88A0758B9FFF726FE094B00224A
:10315000A3F8C021074BDB6813F4803F04D108BDFE
:103160000321FFF799FFF1E700220321034803F051
:103170005FFBF4E72004002020140020FC1A00204C
:1031800000B583B0194B03F58052002182F869170E
:10319000DB6813F0010F08D0B2F8860768B9FFF7B3
:1031A000FBFD124B0022A3F8C021104BDB6813F487
:1031B000803F06D103B05DF804FB0121FFF76CFFEF
:1031C000EFE70B49002381F86937012381F868375D
:1031D000B1F89827C1F8502600930323B1F89A2735
:1031E000B1F894170348FFF751FDE3E720040020EE
:1031F00020140020FC1A002000B583B01F4B03F5FB
:103200008052022182F86817002182F86917DB6872
:1032100013F0010F1ED1194BDB6813F4803F16D059
:10322000174BD3F84C26C3F85026B3F890371BB988
:10323000134B6322A3F89027114900230093032323
:10324000B1F89027B1F894170E48FFF71FFD03B0AF
:103250005DF804FB0120FFF78BFD0120FFF7C4FEA2
:103260000749B1F88237A1F88C3700220092134643
:10327000B1F880170348FFF709FDCCE720040020D0
:1032800020140020FC1A002008B5164BDB6813F050
:10329000010F05D0144BB3F8863783B9FFF7ACFFA5
:1032A000104BDB6813F4803F08D00F4AB2F8982720
:1032B0008AB913F4002F09D1FFF79EFF08BDFFF76D
:1032C0005FFF094B012283F86927E9E700210F20FE
:1032D000FEF70AF9F0E7FFF753FF034B012283F8EB
:1032E0006927EBE7200400202014002038B50546AC
:1032F000FCF752FF044672B6154B93F86837012B62
:1033000001D0032B16D1124BB3F88C379BB2012D91
:103310000ED04FF0FF304FF6FE7200211844FEF73A
:10332000FBFA80B20A4BA3F88C0704B962B638BD29
:103330000120F0E70120FFF71BFD2846FFF754FEB0
:103340000448FFF701FD044BFA22A3F8C021ECE783
:103350002014002008830001200400200F4BDB68AC
:1033600013F0007F03D10E4B93F84406704710B55D
:103370000B4CD4F808381869FEF758FAD4F8083816
:103380001B78022B04D0012814BF0020012010BD9F
:10339000012814BF00200120F9E700BF200400200D
:1033A0002014002030B583B0054601230093032389
:1033B000C5224FF4801118484068FFF765FB0446AA
:1033C000164BDB6813F4002F11D025B903211448E4
:1033D00003F0B4F858B1134B1868FEF727FA012828
:1033E0000AD0114B1868FEF721FA01280CD0B4FA64
:1033F00084F0400903B030BD0122C5214FF4001014
:10340000FFF754FA0124ECE70222C5214FF48000B3
:10341000FFF74CFA0124EAE71C03002020040020F7
:10342000FC1A0020441E0020401E002008B5194B45
:103430005B6A13F0010F20D0164BDB6813F4807F1A
:1034400002D013F4805F0CD0124BDB6813F4803F82
:1034500010D0114B1B8883B1104A1388013313809D
:103460000BE001F087FD0028EED10D4B186803F04A
:1034700000FBE9E713F4003F00D108BD0020FFF78F
:1034800091FF0028F9D100220321064803F0D0F96A
:10349000F3E700BF200400201E040020AA1C002027
:1034A0001C030020FC1A002008B5204BDB6813F435
:1034B000003F02D01D4B1B7803B908BD1C4B586858
:1034C000FFF7ECFA01280ED0194B5B685A6C7AB101
:1034D000B2F90020B3F924309A4219DD154B0222CB
:1034E000A3F89E2704E0134BB3F89C27A3F89E276C
:1034F000104BB3F89E379BB101210D4B1868FFF7B5
:1035000073FC0C4AB2F89E37013BA2F89E37D4E711
:10351000B2F5707FECDD074B0222A3F89E27E7E7A8
:103520000021034B1868FFF75FFCC6E7200400206A
:103530001C03002020140020294BB3F8AC37002BCB
:103540004CD0284901F580504FF0000CA0F8ACC7D2
:103550004FF080431A8892B222F0010292B21A8090
:103560004FF6FF729A849A8B92B222F0080292B2BE
:103570009A83A3F83CC09A8992B222F0090292B2CF
:103580009A81D0F8E0261848A0FB0202920C02EBC8
:1035900042025000013880B2188586229A851A8826
:1035A00092B242F008021A801A8A92B222F0010204
:1035B00092B21A829A8992B242F009029A819A8A48
:1035C00092B242F001029A8201229A871A8892B23C
:1035D00042F001021A800823A1F8C031704700BFF1
:1035E000201400202004002083DE1B4310B5044675
:1035F000FCF7D2FD72B623680133236000B962B6CE
:1036000010BD000008B51B4B1B68112B03D0194BD4
:1036100000221A6008BD184800F580520A23A2F85B
:10362000A837164B93F803C0197941EA0C21A2F888
:10363000A01793F805C0997941EA0C21A2F8A217C6
:1036400093F807C0197A41EA0C21A2F8A4175B7B12
:10365000012B14BF00230123A2F8A637436A002BD5
:10366000D5DA064900234B7490F82200FEF73EF8A5
:10367000CDE700BF00040020200400200404002047
:1036800008B520210B48FDF75CFC58B1094B9B881D
:10369000DAB2094B1B68112B05DC0849CA54013307
:1036A000054A136008BD0122C9214FF00070FFF7E1
:1036B000FDF8F7E700380140000400200404002072
:1036C000084B1B686BB1084A128812F0800F08D0B3
:1036D000C3F10C020549895C034A9180013B014A10
:1036E00013607047FC030020003801404494000838
:1036F00008B5154B5B6A13F0040F0ED0124B5A6AD3
:103700006FF382025A6200229A8783F83B2083F883
:103710003A2083F8392083F838200B4B93F8003295
:103720005BB9FDF75FFFFDF75DFF074BDB6813F447
:10373000001F05D103F0D0FF08BD01F07FFDF0E7C9
:10374000FFF7BEFFF6E700BF2004002008B5FFF733
:1037500059FF0D4BB3F8A8371BB1013B0A4AA2F839
:10376000A837094BB3F8A8374BB9074B4FF69D72F2
:10377000A3F8A027A3F8A2270122A3F8A627034BAA
:103780000C221A6008BD00BF20140020FC0300209A
:1037900010B5044600F00F0301209840FCF764FFC9
:1037A000A8B10B4B9B8C9BB25BB10A4AB2F8BC37F9
:1037B0000133A2F8BC37064A938A9BB243F0010357
:1037C000938204F00F040120A040FCF75DFF10BDC0
:1037D000002C01402014002008B5054BDB6813F0D5
:1037E000807F00D108BD0348FFF7D2FFFAE700BF92
:1037F0002004002003B8080008B5054BDB6813F06F
:10380000807F00D108BD0348FFF7C2FFFAE700BF81
:103810002004002019B8000208B50146024B586880
:10382000FFF7E2FA08BD00BF1C03002008B5024BF9
:103830005868FFF733F908BD1C030020044BB3F8A8
:10384000BC27A3F8BE270022A3F8BC27704700BFFF
:103850002014002008B50D4BDB6813F0807F07D1E2
:103860000A4BDB6813F4803F05D1FDF729F808BD4A
:10387000FFF7E4FFF4E7FFF717FE044BDB6813F4F0
:10388000001FF2D0FFF762FFEFE700BF2004002027
:10389000002801DB80B27047404280B270470000D0
:1038A000012808D90A4B03F5805203F5BF53C2F82B
:1038B000DC370020704700EB8000800000F5BF502F
:1038C000034B184403F58053C3F8DC07012070470D
:1038D00020040020022809D040B1012806D00B4B5B
:1038E00003F65C02C3F808280020704700EB800054
:1038F00041F6080303EBC003054A1344043302F501
:103900008052C2F808380120704700BF2014002000
:103910002004002038B50C4BDB6813F0007F00D189
:1039200038BD0A4DB5F80618094C003918BF0121F9
:103930006068FFF759FAB5F8F217003918BF01218E
:103940002068FFF751FAEBE7200400202014002044
:103950001C03002008B50B4B984203D10A4B5B7A3D
:10396000312B07D04069FDF761FF012814BF00200B
:10397000012008BD4069FDF759FFB0FA80F0400909
:10398000F7E700BF7C1C002020040020F8B59A4B0C
:103990001A6B002A65D019465B6B643B4B63002BA6
:1039A0005FDC4A634B6A13F0010F5AD04B68002B5F
:1039B00057D100242546D1F8FC30002B52D0B3F962
:1039C0001C3063F30F048C4BDB6813F0010F59D0EC
:1039D0008A4A5268918961F31F4413F0100F47D04F
:1039E000854BD3F80031002B3FD0B3F91C3063F383
:1039F0000F05824B1B689B8963F31F457E4BDB6978
:103A000013F0040F40F0EE807B4B5B6A13F4804FA1
:103A10000DD0794BD3F8FC3013B1DB8A63F30F057B
:103A2000754BD3F8003113B1DB8A63F31F452B4686
:103A3000224602214020FDF72DFD6F4B9A6A704B04
:103A4000A3FB0213DB0803EB8303B2EB430F08D1A4
:103A5000694BD3F8C43123B1674B4FF00042C3F830
:103A6000C421F8BD4FF49673ABE74FF49673BEE7ED
:103A70006449D06C04F0BAFC04F0A4FE80B260F398
:103A80000F05BBE713F4807F19D05C4A5268928916
:103A900062F31F4441F210021342AFD0564BD3F8E9
:103AA00000314BB1B3F91C3063F30F05534B1B6866
:103AB0009B8963F31F45A1E74FF49673F4E713F472
:103AC000001F23D0504BB3F8A02762F31F44B3F874
:103AD000A22762F30F05B3F8A6770FB14FF4804722
:103AE0004A4B1868FDF7A2FE4603B6B23E43484B68
:103AF0001868FDF79BFE03039BB233439BB2424A17
:103B0000B2F8A427134363F31F4577E713F4A01F0C
:103B100010D0404B1B8863F31F44374B03F5805292
:103B2000B2F8902762F30F05D3F800315B8B63F393
:103B30001F4563E713F4800F13D113F0807F23D167
:103B400013F0007F30D113F4000F3FF457AF2B4B2D
:103B50001A68928962F30F045B689B8963F31F44C0
:103B60004CE7294BD3F8943763F30F0403212A4819
:103B700002F0E4FC60F31F44204B5B68586BFDF7D8
:103B800065FE60F30F0539E7FFF750FE60F30F04A1
:103B9000224E0321304602F0D8FC60F31F44B6F8F1
:103BA0009E3063F30F0529E71D48FFF7D3FE60F34E
:103BB0000F04114B03F5805292F8F5172C2000FBEF
:103BC0000131B1F8621061F31F4492F8E11700FB74
:103BD0000133B3F8623063F30F05B2F85E3863F374
:103BE0001F450BE701F0BAF9401160F30F0501F032
:103BF000BBF960F31F4507E7200400201C030020E9
:103C0000CDCCCCCC0000C84220140020441E0020A3
:103C1000401E00201E040020FC1A0020401B002033
:103C20007C1C002010B501460D4B03F5805C9CF810
:103C3000C0079CF8F5E72C2404FB0E3EBEF9622079
:103C40009CF8E1E704FB0E33B3F96240BCF85E3840
:103C500043EA044342EA40524020FDF71BFC10BDFA
:103C60002004002010B508214FF08040FDF7CDF86A
:103C700090B1AB4BDB6813F4800F08D0A94BD3F89D
:103C8000B037002B03DD4FF0804300229A870821D4
:103C90004FF08040FDF7C5F801214FF08040FDF75F
:103CA000B4F8002800F04D819D4BDB6813F0010F44
:103CB0002FD09C4BB3F88C379BB253B3984B5B6AB5
:103CC00013F0080F10D1964B93F8103163B9944B51
:103CD0005B6A13F0805F04D0924B93F86837022B35
:103CE00002D09148FFF730F88E4BB3F88C379BB277
:103CF0004FF6FF7293420CD08A4AB2F88C379BB2CF
:103D0000013B9BB2A2F88C37B2F88C379BB2002BE8
:103D10005FD0834BDB6813F4800F13D0814BD3F853
:103D2000B037002B0EDD013B7E4AC2F8B037002BC6
:103D30006EDD4FF080420123938713889BB243F0DE
:103D400001031380764BDB6813F0007F00F0F480F2
:103D5000744BB3F8C837002B00F0EA80714B93F82E
:103D6000CF37042B59D16E4B03F58052D2F8DC27A4
:103D700052782C2101FB023393F86C30002B6DD06C
:103D8000684B93F8C43713F0040F67D0654B93F872
:103D9000D8375BB962492C2000FB0210B0F96200F1
:103DA00001F58051B1F8D61788420DDB012B55D1B2
:103DB0005B4B2C2101FB0232B2F9622003F58053E8
:103DC000B3F8D6379A4249DD564B0122A3F8C827EB
:103DD00044E000214FF08040FCF7BFFF514B93F8C7
:103DE0006837012B04D04F4B002283F8682790E7F7
:103DF0004C4B93F8693723B94A4B002283F8682764
:103E000087E7484B002283F86927FFF7F5F980E739
:103E1000444B0122A3F8AC2794E7424CD4F808386D
:103E2000D868FEF791FF94F8CD37062B32D0042BDB
:103E300030D03C4B93F8CF37052B40D03949D1F8DF
:103E400008385A88986802445A80D1F808381A7895
:103E5000022A03D05988DA8B91425ED0314AB2F8F7
:103E6000C837013B9BB2A2F8C837002B64D1144677
:103E7000012382F8CB3700212C48FCF76EFF94F821
:103E8000CA37002B58D00A20FFF7CCFE002284F856
:103E9000CA2751E0234BD3F80808FFF75BFD20B198
:103EA000204B0122A3F8C827C8E71E4BB3F8C83738
:103EB000012BC3D11B4B002283F8CC27BEE7194B43
:103EC00093F8C43713F0040FB8D0164BD3F8082872
:103ED0005288B3F8D2379A42B0D1124B93F8C03718
:103EE000052B0ED0062B12D00D4B03F58052D2F8C5
:103EF000DC2752782C2101FB0233002283F86C204E
:103F00009CE7084BD3F8DC3764225A82ECE7054B78
:103F1000D3F8DC3700225A82E6E700225A809DE778
:103F2000200400202014002008830001002C014000
:103F3000044B0022A3F8C82701214FF08040FCF772
:103F400070FF10BD2014002070B50E461546244B9E
:103F5000D3F80838DA8B824200D2104693F800C0BA
:103F6000BCF1020F04D05988814220D8441A01E0E4
:103F70005A88841A1B7923B9194B93F8C037012B3F
:103F800026D1DCB1BCF1020F14D0E043C00FFFF723
:103F90002BF82046FFF77CFC114CA4F8C8073146EB
:103FA00004F2DC60FEF7C4FE84F8CA5770BD091A3B
:103FB000541ADFE70120FEF7DBFEE6E7084B01229B
:103FC00083F8CB27002DF1D00A20FFF72BFEEDE779
:103FD000034B002283F8C0270B20FFF723FEE5E701
:103FE0002014002008B5494A92F8CE3782F8CF371E
:103FF000591E82F8CE17062B28D8DFE803F07E760C
:104000005951453B0400414B93F8C037052B07D06D
:10401000062B1CD03D4B47F6FE72A3F8D22711E0C9
:104020003A4BD3F8DC275188A3F8D0179188A3F82E
:10403000D217D188A3F8D4171289A3F8D627012262
:1040400083F8D827314B012283F8CB2708BD2F4BAB
:10405000D3F8DC275189A3F8D0179189A3F8D21798
:10406000D189A3F8D417128AA3F8D627002283F89F
:10407000D827E7E7254BD3F808180022C98CB3F8F6
:10408000D007FFF761FFE1E7204BB3F8D427A3F88F
:10409000C8274FF47A7103F2DC60FEF749FED5E7DA
:1040A0000820FFF7BFFD194B012283F8CB27CDE78E
:1040B000164B93F8C43713F0080F07D1134B0022A7
:1040C00083F8CE27012283F8CB27BFE70F4B93F865
:1040D000C4276FF3C30283F8C427D3F8083800223B
:1040E000998C988BFFF730FFB0E70920FFF79AFD16
:1040F000064B012283F8CB27A8E7044B002283F864
:10410000C0270A20FFF78EFDA0E700BF2014002083
:1041100070B504460E461546244BD3F80838187877
:10412000022816D0002C21DBACB302282FD0E043AC
:10413000C00FFEF759FF2046FFF7AAFB1B4CA4F85F
:10414000C807314604F2DC60FEF7F2FD84F8CA5776
:1041500070BD5A88A118DB8B994202DD9B1A1CB2F4
:10416000E2E70029E0DA524214B2DDE7624212B21D
:10417000DC8B92FBF4F304FB1322012B02DD131EF4
:1041800018BF012303FB0444A41A24B2CCE7012086
:10419000FEF7EEFDCBE7054B012283F8CB27002D80
:1041A000D6D00A20FFF73EFDD2E700BF2014002042
:1041B000F8B57E4BDB687E4A1A420BD07D4BD3F8B4
:1041C00074273AB11946D3F878370A3BC1F87837E3
:1041D000002B00DDF8BDC1F87827774B1868FDF794
:1041E00025FB0646B0FA80F46409744B1868FDF7A5
:1041F0001DFB0746B0FA80F56D090EB9002855D0B1
:104200006A4BDB6813F0010205D06A4991F8681720
:10421000042903D011B113F4807F7FD00EB1002F99
:104220006DD1644B93F868374BB9002A44D1614B88
:10423000B3F86C27A3F87227042283F86827002FAD
:104240003ED0002E49D0594F07F58055B5F872176A
:10425000B5F86C07FDF75AFB81B2A5F87217FB6839
:1042600013F0010F3ED1514BDB6813F4807F0DD06A
:104270004E4B03F58052B2F872275B6A13F4007F4D
:1042800039D0234603214020FDF704F9494CB4F806
:104290007207B4F86E37184480B2A4F87207B4F805
:1042A0007017FDF72DFBA4F8720793E70622C521CE
:1042B0000220FEF7FBFA8DE70120FEF759FDB6E775
:1042C000FFF74CF80028BCD13A4BB3F86C27A3F8A1
:1042D00072272846FEF788FEB5E7FFF73FF801286A
:1042E000B1D1F1E74FF6FF72A5F88C2705F2DC603B
:1042F000FEF71EFDB7E7331E18BF0123C2E722B148
:104300002C4B93F86837042B05D02A4BB3F86C2755
:10431000A3F872275EE7FEF73FFDF6E713F0007F94
:104320003FF458AF234B93F8C037002B7FF452AFC4
:1043300016B1002F7FF44EAF0220FFF7CBFA1D4BD2
:10434000B3F8C837C3B91B4BB3F86C37194AA2F896
:104350007237DC08B2F8C827CAB9164BB3F86C2715
:10436000A3F8722706B964420022124BB3F8721701
:1043700020B2FFF7CDFE2DE70E4BB3F87207D3F84E
:104380000838D98CFA30FDF7BBFA83B2DEE7094D65
:10439000B5F86E07184480B2A5F87207D5F808384A
:1043A000D98CFDF7ADFAA5F87207DBE720040020F1
:1043B00001010002201400205C1E0020581E002075
:1043C00038B5444A92F8CC3782F8CD37591E82F876
:1043D000CC17062B19D8DFE803F0745A433426199A
:1043E00004003C4CD4F8083800251D710120FEF76C
:1043F000BFFCD4F8083847F6FE725A80D4F8083863
:104400002A46198C3448FFF783FE38BD314BD3F868
:10441000081800224A80D3F80838D98CB3F91A005A
:10442000FFF776FEF1E72B4BD3F8082847F6FE712D
:104430005180D3F808380022598C2748FFF768FECE
:10444000E3E7244BD3F80828118B5180D3F80838C0
:10445000188B40420022598C00B2FFF759FED4E776
:104460001C4BD3F8082800215180D3F808280121DB
:10447000117193F8C43713F0080F03D1154B0022C4
:1044800083F8CC27134B012283F8CB27BDE7114BD0
:1044900093F8C43713F0080F04D10E4B012283F8B0
:1044A000CB27B2E70B4B93F8C4276FF3C30283F813
:1044B000C427D3F808380022998C988BFFF744FD65
:1044C000A3E7044B002283F8C0270A20FFF7AAFBCA
:1044D0009BE700BF201400200280FFFF08B5134BAC
:1044E000DB6813F0007F1FD0114B93F8C037BBB1CE
:1044F0000F4A92F8CB27BAB10D4A002182F8CB17A8
:10450000012B05D0022B06D073B1FFF76BFD0BE03A
:10451000FFF756FF08E0064B002283F8C02703E0B0
:10452000034B002283F8CB2708BD00BF20040020E6
:104530002014002070B5044600250BE01048FDF75C
:104540001DF964000F4E3046FDF723F93046FDF7A4
:1045500015F901351F2D05DC002CEFDA0848FDF7B1
:1045600018F9EEE7084C2046FDF713F90448FDF76B
:1045700005F901F0ADFE2046FDF700F970BD00BF62
:1045800002830400038308000A83000408B52C4B4F
:10459000D3F85036002B23DD294A92F86827022AE7
:1045A0001FD0013B2649C1F85036002B18DCA1F57D
:1045B0008053DB6813F4803F2ED0012A19D0FEF718
:1045C000EBFB204BDB6813F0007F09D01C4BD3F8CA
:1045D00050362BB1013B1A4AC2F85036002B26DD6B
:1045E00008BD1749D1F84C0641F60A218842D8D1B6
:1045F000F6E791F86927002AE1D013F4002F06D1DD
:104600000F4B002283F86927FEF7F6FDD7E700215C
:104610000F20FCF769FFF3E713F4002F02D1FEF738
:10462000BBFBCEE700210E20FCF75EFFF7E7002082
:10463000C2F85006FFF77EFF0A20FFF7F3FACFE734
:10464000201400202004002010B5094B5B6A13F0F1
:10465000010F04D102F01EFAFFF798FF10BD054CC0
:104660002068FEF711FC6068FEF70EFCF4E700BF5F
:10467000200400201C03002008B501213048FCF76D
:10468000C4FB08B32F4BDB6813F4803F09D02E4ADC
:10469000D2F850262AB1013A2B49C1F85026002AF7
:1046A00013DD284BDB6813F0007F09D0264BD3F8CD
:1046B00050362BB1013B244AC2F85036002B35DD71
:1046C00001211F48FCF7ADFB08BD0A460021C2F8D6
:1046D000501692F86827012A05D013F4002F20D134
:1046E000FEF75AFBDDE7184A92F86927002AD8D06E
:1046F00013F4002F11D1134B03F58052002182F8DF
:104700006917DB6813F4803F04D013464EF660222D
:10471000C3F84C26FEF770FDC3E70F20FCF7E4FE5C
:10472000E9E700210E20FCF7DFFED9E70020C2F800
:104730005006FFF7FFFE0A20FFF774FAC0E700BF3C
:10474000002C01402004002020140020094B45F2D9
:1047500055521A6006225A60C0EB401200EB8200EC
:10476000400080B298604AF6AA221A604CF6CC4209
:104770001A6070470030004010B500243D4B1C60AB
:1047800021464FF00060FCF7E9F84FF44070FCF769
:104790009FF80A20FFF7DAFF02F08EFB02F09AFB87
:1047A00002F056FD02F076F9012002F0D5FC02F08D
:1047B00025FA022002F0D0FC03F03AF8032002F0C0
:1047C000CBFC01F063FE02F0D9FE00F0B3F900F07B
:1047D0005DFA2948FCF7F4FF80210846FDF750FBFD
:1047E000264B1B68264AA2FB03231B0A013B4FF002
:1047F000E0225361234BF02183F8231094610723B7
:1048000013610DE02048FDF7D3FA02E01F48FDF7E1
:10481000CFFA1F4B1B882BBB164B1B68002BACD150
:10482000144B1B68002BA8D11A4803781A4AA2FB24
:10483000031202F0FE0101EB52029B1ADBB203707D
:10484000012BE3D0022B09D0002BE2D1134B1B7AB2
:10485000412BD7D01248FDF7ABFADAE71148FDF744
:10486000A7FAD6E780210846FDF70AFB084B00228D
:104870001A80D1E7180400201983000200000020EC
:10488000D34D621000ED00E03C01002064000020E8
:10489000A81C0020AC1C0020ABAAAAAA200400205F
:1048A0002C0200201C00002008B503F061F808BDB0
:1048B00008B5B1F5805F08D20023202B0EDC32F85A
:1048C00023C08C450AD20133F7E713460822C221E0
:1048D0001848FDF7DCFF4FF0FF300BE0022805D051
:1048E000032824D13BB9B2F9020003E002EB8302B2
:1048F000B2F9020008BD03F18040013802EB800CE0
:1049000032F82000091A090402EB830E32F8233032
:104910001B1ABEF90220BCF90200121A91FBF3F334
:1049200002FB03F303F5004300EB2340E2E74FF003
:10493000FF30DFE7EFBEADDE00294CD02DE9F843B4
:1049400005460E4600241F2C06D835F82430B34205
:1049500002D20134A4B2F6E705EB840135F8243025
:10496000B34233D040F6FE7293422FD80CB1013CD3
:10497000A4B204F1010905EB8903B3F9020005EBC8
:104980008403B3F90270C01B03F0DCFC804635F8E9
:10499000290035F82450401B03F0D4FC0146404662
:1049A00003F0D8FD0446701B03F0CCFC214603F055
:1049B0001DFD0446384603F0C5FC214603F00EFCFD
:1049C0004FF0745103F012FDBDE8F883B1F9020015
:1049D00003F0B8FCF8E700207047000070B5474BC3
:1049E0001D882C23464C03FB0544464B1C60464B5C
:1049F00033F81510E182454A138804EB43004180E7
:104A000001339BB21380092B3FD900224FF0004C99
:104A10006FF00041104600E00132092A0BDC04EB84
:104A20004203B3F902301844994200DD19469C450F
:104A3000F2DA9C46F0E76144401A40F3CF0060830D
:104A400003F080FC324B196803F0D0FC2062042D87
:104A50000ED8DFE805F0031B310D3700B4F91A005A
:104A600003F070FC2B4B196803F0C0FC2A4B186054
:104A7000264B00221A80214A138801339BB21380EF
:104A8000052B02D9134600221A8070BDB4F91A40D2
:104A9000A4B2224E21463046FFF74EFF204B18604D
:104AA000204DC5F8AC01324621460320FFF700FF38
:104AB000D5F8FC309883DBE7014603F08FFB1A4BF7
:104AC0001860D5E7B4F91A10184A89B20220FFF726
:104AD000EFFE83B2164A1380092B04D8114BFE2235
:104AE00083F82220C4E7642B04D90E4BFE2283F8FE
:104AF0002220BDE70B4B83F82200B9E7BC1D002044
:104B0000B41C0020B01C0020D41D0020BE1D0020BD
:104B1000300300202C030020CC1D00204895000805
:104B2000D01D002020040020C81D00205094000843
:104B3000C41D002030B593B001214FF40370FBF782
:104B40008DFF01210846FBF77BFF4FF40040FBF788
:104B50000FFF1B23ADF8443000248DF8474011A906
:104B60004248FBF735FE0223ADF8443011A9404816
:104B7000FBF72EFE0C9401258DF834508DF835503E
:104B80004FF460230E930F9406238DF84030394C78
:104B90000CA92046FBF7BAFB29462046FBF7DCFBB5
:104BA0002046FBF7EFFB3348FBF7F1FB0028FAD177
:104BB0003048FBF7F4FB2F48FBF7F6FB0028FAD14F
:104BC0002C4C0523012200212046FBF700FC052385
:104BD000022201212046FBF7FAFB0523032211469E
:104BE0002046FBF7F4FB0523042211462046FBF781
:104BF000EEFB05231A4609212046FBF7E8FB0723B5
:104C0000062210212046FBF7E2FB1B48FBF736FC8F
:104C10001A4B01931A4B029300230393062204922A
:104C20000593802206924FF4807207924FF48062BF
:104C30000892202209924FF400520A920B93114AD3
:104C4000936811490B6023F4FF4323F070030B605A
:104C500043F4165343F020030B609360049BD3602E
:104C6000019B1361029B536113B030BD00080140EA
:104C7000000C014000240140080002404C24014087
:104C8000D41D002000000240C01D002010B50121ED
:104C90000648FBF787FC064C01212046FBF767FB23
:104CA00001212046FBF788FB10BD00BF0800024031
:104CB0000024014008B55C210148FCF7D7FD08BD80
:104CC000E01D002038B501221146104601F074FEA7
:104CD0000368064CA3650025A5640548FCF770FD34
:104CE000012384F856306561237038BDE01D002033
:104CF0000AC8000408B54FF48060FBF7B5FCC8B1E2
:104D00000F4B93F84730292B10D80D498A6D928CA0
:104D100092B2C96C511AFD290DDD09491944FE20D2
:104D200008760749CA64013381F847304FF4806040
:104D3000FBF7AAFC08BD024818440176F1E700BF62
:104D4000E01D002038B57F4B93F85630002B45D03E
:104D50007D4BDB6913F0040F35D07A4A936C013335
:104D60009364C82B17D0C92B39D0B3F5967F38D0B0
:104D700040F2E512934200F0D780B3F5FA7F22D1DA
:104D80000021704B9964704B93F8B42161F3410298
:104D900083F8B42117E06D48FCF712FD13E0694A6F
:104DA0001A44FF2111760133DBB2292BF7D9654A6A
:104DB000002382F84730D364926D93846448FCF7F3
:104DC000FFFC01F0B3FA5F4B5B693BB95D4B6FF0E1
:104DD00062021A654FF2A032A3F8542038BD0023B6
:104DE000E3E7FBF7EDFB002306E0564A1A440021F7
:104DF00082F842100133DBB2042BF6D9002423469B
:104E000002E001240133DBB2272B1DD84FEAD30E79
:104E10004C4901EBD30090F842205200D2B280F806
:104E20004220981C0144097EA1F13300C0B2312810
:104E3000E8D96539C9B23B29E3D84249714442F007
:104E4000010281F84220DDE784B93E4A92F842002F
:104E500092F84310431892F844E0734492F845C026
:104E60006344DBB292F84620934203D0354B0022D4
:104E70005A61A8E7334B01225A611B78934205D04F
:104E8000022B28D02F4B00225A619CE741EA0020D8
:104E9000304B83FB002080104FEA0E2404F4FE44C4
:104EA0004CEA0404640183FB043444F38F041EF0D1
:104EB000800F0ED164220021FCF71AFD214D2865D8
:104EC0004FF47A6224492046FCF712FDA5F85400FD
:104ED00079E76442EEE741EA00210812194B1865B0
:104EE0004FEA0E2303F4FE434CEA030C4FEAEC03B3
:104EF0004FEADC0C134AA2F854C01EF0800F0FD109
:104F00005A221421FCF7F4FC0E4C20654FF4C862C1
:104F10000021B4F95400FCF7EBFCA4F8540052E76C
:104F20005B42A2F85430EBE7064B5B69003B18BFCD
:104F30000123054A92F8B41163F3410182F8B411D8
:104F400041E700BFE01D0020200400200A83000488
:104F50000AC800046766666600FBFFFF014BB3F9F1
:104F600054007047E01D0020014B186D704700BFD2
:104F7000E01D0020014B5869704700BFE01D002074
:104F800000487047341E002030B583B00E4B5B6A7A
:104F900013F4004F03D00425284603B030BD044667
:104FA000FBF778FBA00200F10060FBF7BBFB0546B6
:104FB000FBF77CFB042DEFD0009523460222C32192
:104FC0000420FDF753FCE7E72004002058B9012333
:104FD0000B7005224A7006228A706122CA700B711A
:104FE00020234B717047012800D070470B463122B7
:104FF00003F8012B054AD2F834261068C1F80100E5
:105000009188927999809A71EFE700BF201400206F
:1050100038B504890388C3F30222C3F3C403012A09
:1050200048D008D8002A71D1052B6FD8DFE803F0EB
:1050300014171B1F232A911D01F00701012965D8B0
:10504000032A58D03C4D082B60D8DFE803F0565EA9
:105050006062646C6E707200384B1C7656E0384BA0
:10506000A3F8484652E0204601F038FD4EE0344BAC
:10507000A3F89C474AE0314BDB7D03B1E3B22F4AF2
:10508000D37543E0022C09D0032C0DD0012C3DD167
:105090002A4AD36943F00203D36137E0274AD36930
:1050A00043F00403D36131E0244AD36943F0080399
:1050B000D3612BE0052B29D8DFE803F003070B0FA2
:1050C00013171F4BA3F86C4720E01D4BA3F86E4746
:1050D0001CE01B4BA3F8704718E0204601F022FDAE
:1050E00014E0E0B201F056FD10E0154BC3F8744730
:1050F000C3F878470AE0134DA5E76B68C26823EA56
:10510000020381680A4013436B60AC8438BDEC84B1
:10511000FCE7AC82FAE7204603F010F90A4903F0F5
:1051200019FAE864F2E76C85F0E7AC85EEE7EC8508
:10513000ECE72C86EAE700BF3405002020040020BD
:1051400020140020840500200000C84208B500F0AB
:105150003003302B08D010F0100F08D110F0200FC2
:1051600008D0FEF70DF808BDFEF78EF8FBE7FEF756
:1051700043F8F8E7FDF710FEF5E7000010B5044628
:105180002C4B03F580520A21A2F846165B6A13F4F1
:10519000001F05D0A2F580535B6A13F0010F25D1E3
:1051A000244B5B6A13F0006F2BD0234B0A22A3F829
:1051B000462601231F4A526A12F0800F04D01D4B6D
:1051C0000022C3F8C42101231A4A526A12F0020FC6
:1051D00019D1184A526A12F0804F27D12BB1154AC3
:1051E000536AE16823EA0103536210BD072001F00E
:1051F000B3FF01F04FFC0F4B5A6A6FF355525A62DE
:10520000CEE70023D6E70B4B5A6A6FF300025A62CF
:105210005A6A6FF355525A6203F58052D2F8342617
:1052200012781A7201F096FD0123D2E702F0C8F855
:10523000D5E700BF2004002020140020F0B587B07F
:10524000FCF714FAA8B1B14B0522A3F8BC2193F8DE
:105250000B32C3F3C103012B0DD0022B00F0DE860D
:10526000002B00F0EB85AA4B0722C1218020FDF71F
:1052700028FB07B0F0BDA54BD3F8083203F47E330A
:10528000B3F5123F4BD0A14BD3F80832C3F3C6237A
:105290000D3B402B00F2C985DFE813F0AF01C705D5
:1052A000C70546008B009800A500C705C7059001FB
:1052B000C705C705C705C705C705BC00C705C7059E
:1052C000C7055500C705C705B301C705C705F901DF
:1052D0000F02C705C705C705C7057703B904C7058A
:1052E00050031D051F05C70533054C05C705C70538
:1052F000C705C705C705C705C705C705C705C7054E
:10530000C7055500E601C705C705360239023C024C
:105310003F02420290025F024B02550055007D4A57
:10532000138801331380AEE77848D0F81032D0F8F4
:1053300014120B40426A22EA01021343436200F551
:105340000270FFF71BFF714B5B6A13F4807F90D0F4
:105350006E4B93F82210BDF80A2061F3CA02ADF833
:105360000A209DF80B2042F018028DF80B20D3F88C
:105370000822C2F3C622029962F3D12102919DF85C
:105380000A2042F004028DF80A20B3F80832C3F371
:10539000C703BDF8082063F3CA02ADF808209DF8E2
:1053A0000C306FF303038DF80C3002A8FCF710F8F3
:1053B0005FE7564B93F81002FBF774FE0028C2D14A
:1053C000554991F84400FBF72BFEBCE74F4B93F88F
:1053D0001002FBF767FE0028B5D04F4991F8440052
:1053E000FBF746FEAFE7494BB3F80832C3F3C702F9
:1053F00013F0080F03D0454BD3F81012D96212F006
:10540000020F03D0414BB3F814221A633F4B1A6BBF
:105410005A6398E73D4EB6F80842C4F3C704A700A4
:1054200004EB84052D0105F58875354404352846BF
:1054300001F01FFB96F810223B1906EB031383F8CB
:105440001621736A13F0010F3FF47DAF042A12D8BE
:10545000DFE802F003082038640000212846FDF749
:10546000C3FC70E7294B502202FB043393F8183138
:1054700013F0400F09D1284601F0FBFA0722C5219D
:105480004FF40040FDF712FA5DE701212846FDF7D1
:10549000ABFC58E71D4B502202FB043393F9183143
:1054A000002BE8DA194AB2F81212502303FB042346
:1054B000A3F81C11B2F81422A3F820216422A3F847
:1054C0001E2140E7114B502202FB043393F819319F
:1054D00013F0010FCFD00D49B1F8120202FB0412F4
:1054E000A2F81C014FF07A63B3FBF0F3B1F9160296
:1054F000B3FBF0F31B0CA2F81E31B1F9141201FB3F
:1055000003F3DB0BA2F820311DE700BF20040020CD
:10551000280600203C1E0020EC050020A24B502253
:1055200002FB043393F8193113F0020FA3D09E4B02
:10553000B3F81222502101FB0433A3F81C2193F885
:10554000187117F0100F2AD0974EB6F9140202F016
:10555000F9FE4FF0745102F049FF502303FB04663B
:10556000C6F82C01002317F0200F23D08E4AB2F981
:105570001432502101FB0422B2F93821934210DB8E
:10558000894B502202FB0434B4F93811B3F91402E8
:10559000FCF7A8F902F0D6FEC4F82C01D3E60123EB
:1055A000E1E792B200929BB20822C6210020FDF7EB
:1055B0005DF9E5E7002B3FF4C6AE5CE77A4AB2F846
:1055C0000832C3F3C70303EB8300000100F58870C2
:1055D0001044B2F9104203EB830102EB0111A1F870
:1055E0003041B2F9121203EB830302EB0312A2F86B
:1055F0003211043001F03CFAA5E66C48FFF708FDD3
:10560000A1E6694BB3F8102203F58053C3F8642771
:1056100093F86837022B7FF496AE634B5B6A13F006
:10562000805F7FF490AE604BDB6813F0010F11D107
:105630005D4BDB6813F4803F3FF485AE5C4900238B
:1056400000930323B1F89027B1F894175948FDF758
:105650001DFB78E60022009213465549B1F88017E9
:105660005448FDF713FBE3E74F4D02AC05F5027319
:105670000FCB84E80F0095F82220BDF80A3062F3C2
:10568000CA03ADF80A302046FBF7A2FE5BE6464BA4
:10569000DB6813F0010F3FF456AE434D05F580541F
:1056A000B4F87017B5F81002FCF72AF9A4F88807C7
:1056B000B5F81232A4F88A3745E63B4BDB6813F0A5
:1056C000010F11D1384BDB6813F4003F3FF43BAEC0
:1056D000354BB3F8121203F58052A2F89A17B3F8BB
:1056E0001432A2F898372EE62F4D05F58054B4F801
:1056F0007017B5F81002FCF703F9A4F88407B5F8A1
:105700001232A4F88637DDE7FDF7BEFD1BE6FDF794
:1057100011FD18E6FDF734FD15E6FDF76DFD12E607
:10572000234B93F86837042B3FF40DAEFDF734FBA1
:1057300009E61D4B5B6A13F0805F3FF404AE1A4B21
:10574000DB6813F0010F3FF4FEAD174BB3F808020E
:10575000C0F3C000FDF7CAFDF5E5134BDB6813F499
:10576000003F11D113F4800F3FF4EDAD0E4BB3F8B1
:10577000083203F4FF63002B3FF4E5AD0E48FDF75C
:1057800035FFFDF7D9FEDEE5074BB3F80822C2F37B
:10579000C70203F58053A3F890275209032103F2AF
:1057A000DC6001F045F8CEE520040020280600204A
:1057B00020140020FC1A0020D01B0020B24BDB6814
:1057C00013F0010F16D0B04BB3F8083213F0080FE6
:1057D0004AD1AD4BB3F80832C3F3C70013F0100F32
:1057E00006D0A94BB3F8122203F58053A3F8822701
:1057F000FFF7ACFCA44BDB6813F4803F56D0A24902
:10580000B1F81222A14BA3FB0203D21A03EB5203FD
:105810001B0A9F4A1380B1F8083213F0080F2FD1EA
:10582000994BB3F80832C3F3C70013F0100F06D03A
:10583000954BB3F8123213B1964AA2F8903710F094
:10584000040F2AD0904AB2F8143202F58052C2F8FE
:105850004C3610F0400F24D04FF47A7202FB03F361
:105860008C4AC2F84C361CE0874B03F58054B4F8E0
:105870007017B3F81002FCF743F8A4F88007A8E704
:105880000B4601F58054B4F848261421B3F81002F1
:10589000FCF742F8C4F89407C2E77E4B0022C3F835
:1058A0004C26794B5B6A13F0805F31D0764BDB6816
:1058B00013F0807F3FF447AD774B5B6801229A700D
:1058C000714BB3F8083213F0080F24D16E4BB3F8C4
:1058D0000832C3F3C70213F0100F06D06A4BB3F8B7
:1058E000121203F58053A3F8B41712F0040F1FD15E
:1058F000654800F58051B1F8B427012300930323D4
:10590000120AB1F8B81700F5B950FDF7BFF91AE55A
:10591000FFF71CFCCAE75C4B03F58054B4F848263B
:105920001421B3F81002FBF7F7FFC4F8B807CDE76E
:10593000554BB3F81402FDF76FFFD9E7524BDB6903
:1059400013F0020F3FF4FFAC01F0A0FE4E4BB3F991
:105950001002C0B201F0E8FE01F0F0FE012803D011
:1059600001F0ECFE032808D1474C94F8160201F030
:10597000D1FE94F8170201F051FE01F0DFFE01287C
:105980007FF4E1AC01F0BAFEDDE43F4BB3F808224E
:10599000C2F3C70203F58054C4F8C42793F8103249
:1059A00084F8C03794F8C40700F00300FDF792FFB5
:1059B00094F8C037013B072B3FF6C5ACDFE813F086
:1059C00008002B006E009900C200C20001011A01FC
:1059D000304B93F8C43713F0200F07D02A4B03F550
:1059E0008052D2F80828B3F812321383294B93F867
:1059F000C43713F0400F07D0234B03F58052D2F881
:105A00000828B3F814321384224B062283F8CC27DB
:105A1000FEF7D6FC97E41F4B93F8C43713F0200F22
:105A200007D0194B03F58052D2F80828B3F8123288
:105A30009383184B93F8C43713F0400F07D0124BE1
:105A400003F58052D2F80828B3F81432D384114BEE
:105A500093F8C43713F0200F0CD00B4AB2F812029F
:105A600013F0400F0BD0084BB3F814120122FEF7CD
:105A70006BFA68E4074AD2F80828908BF0E7054BE8
:105A8000D3F80838D98CF1E72004002021F1D49014
:105A90001E040020201400201C030020C24B93F899
:105AA000C43713F0400F07D0C04B03F58052D2F833
:105AB0000828B3F81432D384BB4B93F8C43713F0DF
:105AC000200F0CD0B94AB2F8120213F0400F0BD0DD
:105AD000B64BB3F814120122FEF736FA33E4B24A99
:105AE000D2F808285088F0E7AF4BD3F80838D98CA3
:105AF000F1E7AD4B93F8C43713F0400F07D0AB4B31
:105B000003F58052D2F80828B3F81432D384A64B98
:105B100093F8C43713F0200F0DD0A44AB2F8120244
:105B200013F0400F09D0A14BB3F81412012200B2B8
:105B3000FEF7EEFA07E40020F2E79B4BD3F80838B3
:105B4000D98CF3E7984B93F8C43713F0400F07D084
:105B5000964B03F58052D2F80828B3F81432D38458
:105B6000914B93F8C40700F00300FDF799FE00285D
:105B70003FF4E9AB8C4B93F8C43713F0200F0CD0F3
:105B8000894B93F8C037052B12D0884B03F5805210
:105B9000D2F8DC27B3F8123253810220FDF79AFEC7
:105BA000814B062283F8CE27FEF71CFAFFF7CBBB0A
:105BB0007E4B03F58052D2F8DC27B3F812325380C3
:105BC000EBE7794B93F8C40700F00300FDF768FE9C
:105BD00000283FF4B8AB744B93F8C43713F0040FAC
:105BE00006D06423704AD2F8DC275382FFF7ABBBA0
:105BF0000023F7E76D4CD4F81402FEF79BFCB4F8D1
:105C0000123204F58054C4F85036FFF79CBB674B42
:105C1000B3F80812C1F3C70103F58053C3F8C417E2
:105C200000221EE001F00300022802D008B1012882
:105C300029D15E4C04F5805090F8C40700F00300B1
:105C400002EB8303151D04EB4505B5F8085200EB84
:105C5000800003EB800303F5416304EB4304A5805C
:105C60000132032A3FF76FAB4F4B93F8C4371B0940
:105C7000134113F0010FF3D04B4B93F8C437C3F328
:105C80008103012BCED911F0020FE9D1474C04F565
:105C9000805090F8C40700F00300023B02EB83033E
:105CA000151D04EB4505B5F8085200EB800003EB29
:105CB000400303F53F6304EB43046580D0E73B4AB0
:105CC000D2F8100203F28A4142F821000133FF2B7F
:105CD000F5DDFFF738BB0023F9E7344AB2F80832A4
:105CE000C3F3C7035B00D2F8100203F28A4142F803
:105CF0002100D2F8141203F28B4342F82310FFF76D
:105D000022BB294B4FF4FA42A3F82826D3F83426B5
:105D1000002307E052F8044B03F28A40234941F87C
:105D200020400133FF2BF5DD1F4B0022A3F828266E
:105D3000FFF709BB1D4C04F580534FF4FA42A3F85A
:105D40002826D3F834564FF4807103F50A70FBF718
:105D5000FFF8D4F8102282420FD1144BB3F8080296
:105D6000C0F3C70003F58053B3F83036984211D022
:105D70000026FFF709F9002428E003460F22C1217D
:105D80004020FCF784FD04F580530022A3F8282668
:105D9000FFF76FBA044BD3F828222B689A4201D040
:105DA0000126E6E70026E4E7201400202004002076
:105DB000FAF770FC04F28A42A14B53F822102846ED
:105DC000FAF7D0FCFAF772FC04350134FF2CEFDD52
:105DD0009B4C04F580534FF48071D3F83406FBF7E5
:105DE000B7F8D4F81032834209D1C6B9954B0122D5
:105DF0001A60954B0022A3F82826FFF7A4BAB4F83E
:105E00000832C3F3C7031022C1211046FCF73FFD3F
:105E100004F580540023A4F82836FFF72ABA62223A
:105E200011460220FCF798FDE0E7884B0822C121CB
:105E30004FF48070FCF745FDFFF785BA804C04F500
:105E400002730FCB06AD05E90F0094F82220BDF8D0
:105E50000A3062F3CA03ADF80A309DF80B30022213
:105E600062F3C4038DF80B30082104A8FBF7FEFC95
:105E7000D4F80832C3F3C623352B00F2C780DFE81D
:105E800003F01B212A377989C5C5C5C58BC5C5C592
:105E9000C5C591C5C5C5C5C5C5C5C5C5C5C5C5C5E6
:105EA000C5C5C5C5C5C5C5C5C5C5C5C5C5C5C5C5A2
:105EB000C5C5C595C5C5C5BC614B93F822308DF8E5
:105EC000103044E05E4BB3F8080204A9C0F3C700E9
:105ED000FFF77CF83BE05E4BB3F8E030ADF81030F4
:105EE0004FF48063ADF812304FF0006305932EE05D
:105EF000BDF808306FF3CA03ADF808300BE002A814
:105F0000FBF766FABDF80830C3F3C702013262F34B
:105F1000CA03ADF80830BDF80810C1F3C701012964
:105F200011D80022052AEADC01EB41035B0003F1F2
:105F30000053A3F61803985C02F118036B4403F8AE
:105F4000080C0132EEE70023002B3FF492A902A8CF
:105F5000FBF73EFAFFF78DB9394A1A4492F8C81197
:105F600003F118026A4402F8081C0133032BF3DD25
:105F70000123E9E70023F9E7314A1A4492F8CC11EA
:105F800003F118026A4402F8081C0133072BF3DD01
:105F90000123D9E70023F9E72B4BB3F83036ADF8EE
:105FA0001030D4E7264B5B6A0493D0E7264B4FF4BE
:105FB000FA42A3F82826002417E004EBD4735B1000
:105FC000BDF8082063F3CA02ADF808201C4B04F2A8
:105FD0008A4253F82220049204F28B4253F8223072
:105FE000059302A8FBF7F4F90234FF2CE5DD164B0C
:105FF0000022A3F82826FFF73CB94FF48071124B1A
:10600000D3F83406FAF7A4FF0490A0E70F4B082258
:10601000C1214FF48070FCF754FC98E7084BD3F88B
:10602000083203F47E33B3F5004F3FF422A9074B47
:106030000722C1218020FCF744FCFFF71AB900BFFA
:10604000200400201804002020140020280600202E
:1060500000F7FF1F10B5954B5B6A13F0010F47D097
:10606000924B9A6A02F00102904B93F8B41162F3DA
:10607000C71183F8B411B3F9BE21002AD4BF00229E
:106080000122C9B262F3861183F8B411B3F9BC21BD
:10609000002AD4BF00220122C9B262F3451183F85D
:1060A000B411D3F8C421003A18BF0122C9B262F377
:1060B000041183F8B4115B6A13F0010F26D07B4BF7
:1060C0001B781BB3794BDB68002B1FDB774AD27D33
:1060D000E2B113F0010F41D0754BB3F88C3713F0D8
:1060E000010F0BD1714BB3F9C031ABB3012106E005
:1060F0006E4B93F83B2002F00102B5E701216B4B98
:1061000093F8B42161F3000283F8B421674CB4F929
:10611000BE1101390020FBF7E5FBA4F8BE01B4F97C
:10612000BC1101390020FBF7DDFBA4F8BC01B4F978
:10613000C01101390020FBF7D5FBA4F8C00163684A
:106140004BB194F83B3013F0010F00F0AD80FF220B
:10615000564BC3F8B42110BD0021D0E713F4803FA3
:106160000DD113F0807F2ED113F4807F5AD04F4B86
:1061700093F8B4216FF3000283F8B421C6E74B4BC8
:1061800003F58052D2F85026003A18BF012293F846
:10619000B41162F3410183F8B4110321454800F0C2
:1061A000CDF928B9414BB3F9C03153B1012100E019
:1061B00001213E4B93F8B42161F3000283F8B4212E
:1061C000A4E70021F5E73C4C0321204600F0B6F996
:1061D000021E18BF0122A4F5B95393F8B41162F35B
:1061E000410183F8B4111B7A4B2B0FD0562B8DD164
:1061F0003248FBF71BFBB0FA80F35B092B4A92F89D
:10620000B41163F3000182F8B4117FE72C48FBF767
:106210000DFBA4F5B95393F8B42160F3000283F8A1
:10622000B42173E713F0007F14D113F4000F2ED0C4
:106230001E4B1B7A4C2B7FF469AF01F041FA031E11
:1062400018BF0123194A92F8B41163F3000182F8D0
:10625000B4115BE71B48FDF77DFB144C94F8B43197
:1062600060F3041384F8B4311748FDF773FB94F816
:10627000B43160F3410384F8B4311448FDF76AFB8C
:1062800094F8B43160F3000384F8B4313EE7074B6F
:1062900093F8B4216FF3410283F8B421D2B26FF3C3
:1062A000000283F8B42131E7002251E720040020E6
:1062B00020140020FC1A0020401B002003B8080016
:1062C00019B800027C1C0020541C00202C1C00204B
:1062D00080B483B000AF0023FB7102E0FB7901338F
:1062E000FB71FB790F2BF9D900BF00BF0C37BD46FE
:1062F00080BC70470F2815D8DFE800F008160A0C9C
:106300000E101010101012121212121206207047E6
:1063100008207047092070470A20704717207047EF
:1063200028207047002070470720704710B582B0C2
:106330002D4BDB6913F0040F2AD100242A4BDB68B4
:1063400013F0807303D0284A127A4B2A2FD01BB146
:10635000254B1B7A562B39D0234BDB6813F0807FFB
:1063600004D1214BDB6913F0040F02D001238DF817
:10637000063000238DF804306846FAF72FF904211F
:106380002046FBF79DFA0098FAF77EF902B010BD9F
:106390000A210020FAF778FA4FF4806300930C2367
:1063A0008DF805300A20FFF7A5FF0446C6E709214E
:1063B0000120FAF769FA4FF40073009308238DF86F
:1063C00005300920FFF796FF0446C5E703210020AA
:1063D000FAF75AFA082300938DF805300320FFF7E7
:1063E00089FF0446B8E700BF2004002010B584B040
:1063F000044610216846FBF739FA1A4B9C4229D013
:106400004FF40030FBF738FA4FF416530093002393
:10641000ADF80430ADF80630ADF80830ADF80C300A
:106420000C23ADF80A3069462046FAF7FFFC01213B
:106430002046FAF75DFD0B4B9C4210D0262003212D
:10644000FBF73EFA012240F225512046FAF75EFDA5
:1064500004B010BD4FF48040FBF720FAD4E72520AC
:10646000EDE700BF00380140002200E00A46064B7D
:106470005B6803F00103834204D1511C4FF6FF73A4
:106480009A42F3D1704700BF0064004070B582B0FB
:106490004FF00070FBF7F0F9254C236823F002035E
:1064A0002360236843F0010323600020FFF7DCFF33
:1064B000236823F0B8032360236843F04403236078
:1064C0001C4BE361236823F0010323600120FFF7E5
:1064D000CBFF002408E000230093FF22214614484C
:1064E000FAF746FD0134E4B20D2CF4D9104D012425
:1064F000009400231A4621462846FAF739FD0E4E2D
:10650000002286F8C921009423460D212846FAF777
:106510002FFDF168490E01F002011520FBF7D0F9BB
:10652000224610212846F9F79EFF02B070BD00BF39
:10653000006400400B00120020040020083100EB32
:1065400081004368188880B27047083100EB8101F0
:106550004B681B881B040268928D92B20132B3FB18
:10656000F2F0000A642303FB00F0000A7047000009
:1065700038B50446083100EB81014B68188880B2B9
:1065800001F0DCFE05462368988D80B2013001F0F1
:10659000D9FE0146284601F0DDFF024901F026FF41
:1065A00038BD00BF0000C84210B50C460368988D86
:1065B00080B24FF6FF710130FBF7A2F904FB00F047
:1065C0004FF6FF71C00BFBF79BF910BD2DE970432F
:1065D0000446894690461E464568B5FBF1F5681CA1
:1065E0004FF6FF71000CFBF78BF9C8F80000013083
:1065F000B5FBF0F04FF6FF710138FBF781F9306021
:10660000C4F808906368D8F800200132B3FBF2F3B5
:1066100032680132B3FBF2F3E360BDE87083013905
:1066200003290FD8DFE801F00205080B00683430B9
:10663000704700683830704700683C307047006829
:1066400040307047002070472DE9704785B0044600
:106650004FEA001800EB001341F2506505EB83058B
:106660003A4E3544043544212846FBF7FFF8A04450
:1066700006EB880641F29063F450022C3CD0032CC8
:1066800049D0012C01D0002532E041F2546230495A
:10669000B1504FF0190A4FF400600223012B48D08B
:1066A000FBF7FCF804EB0412284B03EB820341F2E6
:1066B000586228499950DFF8948004EB041608EBDF
:1066C000860641F264632022F25041F28C6346F860
:1066D00003A001A8FAF725FB41F2546A01A956F874
:1066E0000A00FAF715FA012156F80A00FAF77FFBBB
:1066F000284605B0BDE8708704EB0412134B03EB8A
:10670000820341F254624FF0804199504FF01C0ACD
:1067100001200346C2E704EB04120C4B03EB820397
:1067200041F254620C4999504FF01D0A0220012396
:10673000B4E7FBF7A1F804EB0412044B03EB82036C
:1067400041F2586203499950B5E700BF2004002088
:10675000002C014000A24A040004004070B584B03F
:106760001446013A032A46D805461E4641BB4461F9
:1067700021462846FFF753FF04F1080205EB820289
:1067800050606846FAF7D6FA2B69ADF8003001235D
:10679000ADF802300423ADF804300023ADF8063024
:1067A00096B9ADF80830ADF80A30ADF80C30ADF858
:1067B0000E30013C032C1ED8DFE804F0151F2831F1
:1067C0000129D5D18461D3E70223ADF8083008232D
:1067D000ADF80A304FF48073ADF80C304FF400730D
:1067E000ADF80E30E5E769462868FAF7B7F90821F1
:1067F0002868FAF7DCFA04B070BD69462868FAF731
:10680000E5F908212868FAF7D9FAF4E76946286813
:10681000FAF726FA08212868FAF7D9FAEBE7694669
:106820002868FAF767FA08212868FAF7D7FAE2E742
:106830004B1E032B66D870B506460C46154690F8DD
:10684000403013F0020F0CD12F4BDB6813F4003FE4
:1068500022D075B12D4BD3F85036012B10DC00201F
:106860001BE04FF4004200212846FCF703FA85B2F2
:10687000EAE7083406EB8404636800221A802CE0FF
:106880000120FCF78FFD48B3642D00D9642505EB8A
:106890008500400080B200E000201B4BDB6813F451
:1068A000800F0BD0194AD2F85026012A06DD2DB1EF
:1068B000154A526A12F0805F00D1012013F0807FE8
:1068C0000ED104F1080306EB83035B68188073693B
:1068D000A3420BD0B369A3420ED070BD0020DCE709
:1068E00029463046FFF760FE80B2EAE7214630468F
:1068F000FFF73EFEF061F0E721463046FFF738FE35
:106900003062EAE7704700BF200400202014002016
:106910002DE970418BB00E4615469846FFF794FE60
:106920000446066109AB08AA2946FFF74FFE00227C
:10693000ADF81620089BADF81430099BADF818305F
:10694000ADF81A208DF81C2005A92068FAF7E0F8A8
:1069500001212068FAF70FFAE36B012B06D0082B10
:1069600004D025BB20460BB0BDE8708101A8FAF722
:10697000EBF94FF40063ADF804304FF48063ADF8E9
:1069800006300023ADF80830ADF80A30ADF80C3011
:10699000ADF80E304FF48043ADF8103001A92068F7
:1069A000FAF7A9F901212068FAF7F3F9D9E7414686
:1069B0002068FAF7D2F9D5E770B505460C461646B9
:1069C000FFF742FE4368114AA2FB03239A0C0368B7
:1069D00002FB04F4013CA4B21C8503684FF6FF726D
:1069E0009A850268938A9BB243F0010393823146F1
:1069F0000068FAF7B2F905EB051541F2506000EBBB
:106A00008500034B1844043070BD00BF83DE1B4378
:106A1000200400202DE978410446164698460023BC
:106A20000A466021FFF774FF0546434632460021BF
:106A3000FFF794FEB8F1000F14D10022314628462A
:106A4000FFF7F6FE9DF818102868FAF786F904EBB0
:106A5000041441F2506000EB8400044B18440430ED
:106A6000BDE878814FF40042E8E700BF2004002031
:106A7000704708B5002181700122028164224281A1
:106A80008181C1810022826101824182FCF7ACF9DF
:106A900008BD000010B50E4C2068FFF7EAFF6068E3
:106AA000FFF7E7FFFCF778F90A4B03F58051002266
:106AB000C1F84C264FF080418A87DB6813F0807F55
:106AC00000D110BD03210448FFF7B2FEF9E700BF73
:106AD0001C03002020040020401B00200D4BDB681D
:106AE00013F4800F00D1704710B504460A4BA3F889
:106AF000AA07C0F380010948FAF756FEC4F3400123
:106B00004FF4C130FAF750FE04F001010448FAF7DF
:106B10004BFE10BD20040020201400200A82000437
:106B200001820200164BDB6813F0010F27D010B56D
:106B3000144BC3F87C07013807281CD8DFE800F0A5
:106B4000041D1B061B1B1B19002400E00224A108C6
:106B50000D4B1868FAF728FEC4F340010B4B186878
:106B6000FAF722FE04F00101094B1868FAF71CFE3F
:106B700010BD0324EBE70724E9E70124E7E77047AA
:106B80002004002020140020481E00204C1E00205D
:106B9000501E002008B5124BDB6813F0010F0AD01D
:106BA0000138042818D8DFE800F003070B0F1300A2
:106BB0000C48FAF705FE08BD0B48FAF701FEFAE7A4
:106BC0000A48FAF7FDFDF6E70948FAF7F9FDF2E79A
:106BD0000848FAF7F5FDEEE70748FAF7F1FDEAE7AE
:106BE0002004002012C0040012880400129804003F
:106BF000128204001292040012C40400064B03F136
:106C00004802C3F8002103F17402C3F8FC2003F129
:106C1000A002C3F80C2170472004002038B50024DE
:106C200020E0474BDB6913F0040F3AD0FEF7A8F9D8
:106C300004EB8402424B03EB0213C3F8580107E054
:106C400004EB84023E4B03EB02130022C3F85821ED
:106C50003B4BDB6813F4003F03D03A4B5B68AB421D
:106C60002DD00134012C40DC04EB84052D0105F509
:106C70008875334B1D44043504EB840203EB021387
:106C8000A3F814414FF49672A3F83021A3F83221EF
:106C900093F8193113F0020FDAD02A4B1B68AB427C
:106CA000BFD0274BD3F8FC30002BC9D01C3304EBEA
:106CB0008401234A02EB0112C2F85831C8E7204B85
:106CC000D3F8FC3043B11C3304EB84011C4A02EBC3
:106CD0000112C2F85831C4E704EB8402184B03EBED
:106CE00002130022C3F85821BBE7164A1368052196
:106CF00059634FF0FF319963D963022083F8400054
:106D00005268D16382F840000D49C96841F2100011
:106D1000014208D00C48D863012083F840000B4B97
:106D2000D36382F8400011F4005F06D0084B1B6863
:106D300053634FF0FF33936338BD10235363F8E779
:106D4000200400201C030020168340000A83000456
:106D5000601E002008B53B4B0122DA751B7AA3F1B7
:106D60003002292A39D8DFE802F04343431717439A
:106D700043434343381F1F1F2121211F2C29292C46
:106D80002C1B1B1B1D322C35171717171717352FE8
:106D90003243191500212CE003212AE02A4928E07A
:106DA0002A4926E02A4924E02A4922E0254B5B7A39
:106DB000312B38D0302B38D027491AE04FF48201DC
:106DC00017E04FF4000114E04FF0814111E04FF063
:106DD00080710EE04FF000710BE00622CA21002006
:106DE000FBF755FD174B0022DA754FF0004100E02C
:106DF0001A49144B5B7AA3F13002D2B2042A16D896
:106E0000104B1B8943F24702934207D043F24812CA
:106E1000934203D043F24912934201D141F400510D
:106E2000084BD96008BD0E49E3E70E49E1E70722A8
:106E3000CA210020FBF72BFD024B0022DA754FF030
:106E40000041DDE720040020110000400005004063
:106E5000001100400000074000000B40050000400A
:106E600000001B4000002B4008B5A0F13003072BA9
:106E700014D8DFE803F008061D040D0A0D10512098
:106E800008BD6420FCE7A820FAE74FF48060F7E72C
:106E90004FF4A060F4E74FF4A060F1E70346082246
:106EA000CA210020FBF7F3FC0020024BD875E7E76E
:106EB0005220E5E72004002008B541F68801044887
:106EC000FAF7D4FC00F0A2FBFDF7F4FE08BD00BF0A
:106ED000200400202DE97841914B1A684FF0FF36CD
:106EE000566396635B685E639E638E4BB3F8E020E7
:106EF00093199BB28C4D05F58054A4F830369B0253
:106F000003F10063C4F83436023A92B2A4F838268A
:106F1000920202F10062C4F83C264FF48068C4F883
:106F200040861A782A725A786A7298782875FFF71C
:106F30009BFF2861D4F83436DA786A751B79AB7513
:106F4000FFF708FFFE2385F82230C5F8C861C5F8B1
:106F5000CC61C5F8D061C4F864876423A4F84636D0
:106F60004FF47A722A636A631E22A4F89C27C4F83D
:106F70007437C4F878376D4BC4F818386C4BC4F8C4
:106F8000403803F578030533C4F86838694BC4F812
:106F90001C38C4F84438684BC4F86C38A3F1F87353
:106FA000A3F60523C4F8203803F1F8731533C4F8A9
:106FB0004838A3F1E073033BC4F87038022384F827
:106FC000F537012384F8E137002412E0E5B22846C2
:106FD000FCF780FC594BD3F808281570D3F8081833
:106FE00000224A80D3F808381A710120FBF7FCFF11
:106FF0000134022CEADD002308E003EB83014A4A56
:1070000002EB810202F5BF5213700133012BF4DD54
:10701000DFF8148108F580531422A3F874284FF484
:10702000FA72A3F8762841F63801A3F8781843F2EB
:107030007001A3F87A184FF47A61A3F87C184FF422
:107040007A70A3F87E08A3F88018A3F882184FF08E
:107050000A0CA3F824C84FF44876A3F82668002049
:10706000A3F828084FF44864A3F82A484FF4C865E9
:10707000A3F82C58A3F82E68A3F83058A3F8324888
:1070800042F6E06EA3F8E2E741F65831A3F8E417C0
:10709000A3F8E62740F2DC51A3F8E817A3F8EAE7E3
:1070A00042F2107EA3F8ECE7A3F8EE27A3F8F0175E
:1070B000A3F84CC8A3F84E68A3F85008A3F85248A8
:1070C000A3F85458A3F85668A3F85858A3F85A4898
:1070D0004FF4C874A3F8F64741F21855A3F8F857CF
:1070E000A3F8FA27A3F8FC17A3F8FE474FF4166499
:1070F000A3F80048A3F80228A3F80418FCF7D0FB73
:107100000220FCF7E7FB98F808304C2B01D0BDE8D3
:107110007881032000F082FA012000F0FBFAF6E704
:107120001C03002000F7FF1F200400200A83000436
:10713000038308000283040009C200022014002017
:10714000044B93F8B4216FF3030283F8B4210122B6
:107150001A7070472004002010B50446042813D08C
:10716000052819D0022807D0FEF774FF124B83F8C8
:107170008748072C1CD010BD104A92F8B43143F058
:10718000010382F8B431EFE70C4A92F8B43143F0CE
:10719000040382F8B431E7E7084991F8B431C3F346
:1071A000C00282F0010262F3C30381F8B431DBE76D
:1071B000FFF7C6FFDFE700BF2014002020040020F7
:1071C000204B1B7E032B3CD01E4BDB6813F0806FE3
:1071D00037D130B583B013F4807F2ED05A220123EB
:1071E0000093002302211848F9F7C2FE154BDB6813
:1071F00013F4807F23D05A23124C84F8CA3194F8B8
:107200002230124DA5FB0323DB0803EB83035A0056
:1072100001230093002302F0FE0203210A48F9F73C
:10722000A7FE94F82230A5FB0353DB0803EB83038E
:107230005A0084F8CB2103B030BD6422CFE7642329
:10724000DAE770472004002000640040CDCCCCCCAD
:1072500008B51D20FAF722FB214B5A6822F0E062A4
:107260005A605A6842F000725A604FF4C130FAF71F
:10727000A7FA1C48FAF7A4FA1B48FAF7A1FA1B4828
:10728000FAF79EFA1A48FAF79BFA1A48FAF798FAA8
:107290001948FAF795FA1948FAF792FA1848FAF7DE
:1072A0008FFA1848FAF78CFA1748FAF789FA17484C
:1072B000FAF786FA1648FAF783FA1648FAF780FAC8
:1072C0001548FAF77DFA1548FAF77AFA1448FAF7EA
:1072D00077FA1448FAF774FA1348FAF771FA08BD06
:1072E0000000014001C00200029B040003C008002E
:1072F00004C010000A8200040BB800080C9B0010A8
:107300000F92008013920800149210001592200032
:1073100011C0020016B8400018B8000117B880006C
:1073200010820100058220001983000210B584B08C
:10733000174BDB6813F4002F06D0154A126912F0C0
:10734000400F21D1002400E0002413F4800F04D06A
:107350000F4B1B6913F0400F18D18CB10C4B5A7AAC
:10736000197D587D0290019100921B7A0322CA2157
:107370004FF40000FBF744FA14B1054B0022DA7514
:10738000034BD87D04B010BD0124DEE70124E5E7FE
:107390002004002010B50120FFF756F9044690F8AC
:1073A000403043F0040380F840304FF47A71FBF72B
:1073B000BFFC022194F83800FAF782FA10BD0000F1
:1073C00010B582B0FFF7FCFEFFF7B0FF002800F019
:1073D000C980FFF723FC654BDB6813F0010F26D152
:1073E000624BDB6813F4803F40D1604BDB6813F0E5
:1073F000807F7ED15D4BDB6813F0007F40F093808F
:107400005A4BDB6813F0007F0AD1584B1B7A552B7F
:1074100000F09F80554BDB6913F0040F40F09F8014
:107420000620FFF799FEFFF735FB02B010BD1020D4
:10743000FFF778FB0120FBF7D7FD0220FFF704F9E7
:1074400090F8403043F0010380F84030DBB243F065
:10745000040380F84030022190F83800FAF730FA3F
:10746000012210214248F8F7FEFFB9E7FFF792FF2B
:107470003E4BDB6813F4003F1DD001230093002333
:1074800003224FF47A710220FFF7C4FA90F84030DB
:1074900043F0020380F84030344BDB6813F4001FE4
:1074A00023D1012210213248F8F7DDFF314B0122B0
:1074B000A3F8AC2799E701230093002303224FF49C
:1074C0007A710220FFF7A6FA90F8403043F00103EA
:1074D00080F84030DBB243F0040380F840300321F1
:1074E00090F83800FAF7ECF9D6E72348FEF77EFF6C
:1074F000D7E701224FF496711046FFF75DFAFEF7C9
:1075000015FF01240094002303224FF47A711046E2
:10751000FFF780FA0094002303224FF47A710220CF
:10752000FFF778FA66E7FFF735FF0220FFF78CF8E0
:1075300090F8403043F0010380F84030DBB243F074
:10754000040380F84030022190F83800FAF7B8F9C7
:1075500056E7064AD36943F00403D3615AE7FDF7BF
:10756000B1FB5DE70820FFF7F7FD5CE72004002092
:10757000006400402014002000380140224BDA69EA
:1075800042F00102DA619A6942F004029A619A6952
:1075900042F001029A61A3F584331A6822F4706202
:1075A0001A601A6842F430621A604FF080438C22ED
:1075B0001A8540F2E7329A859A8B92B222F07002D5
:1075C00092B29A839A8B92B242F060029A839A8B1B
:1075D00092B242F008029A831A8C92B242F48072FC
:1075E0001A841A8C92B222F4007292B21A84012286
:1075F0009A871A8892B242F080021A801A8892B250
:1076000042F001021A8070470010024008B51421B0
:107610000148FAF72BF908BD641E0020052828D878
:10762000DFE800F00312161A1E22124B124A1A61EA
:1076300010B5104C2069FAF7C3F82069FAF780F802
:10764000A060638AA38110BD0A4B0C4A1A61EFE760
:10765000084B0B4A1A61EBE7064B0A4A1A61E7E747
:10766000044B094A1A61E3E7024B4FF4DC321A611A
:10767000DEE77047641E002003B8080002B804006B
:1076800016B840000AB8000401B80200014B0122FC
:107690009A737047641E0020024B00221A709A737E
:1076A000704700BF641E002010B504460121F9F7A1
:1076B0001BFF0C2C00D110BDFFF7EEFFFBE7000015
:1076C000044A93689B6891890B405068181A18BF48
:1076D00001207047641E002008B5074B9B7B13B147
:1076E000054B1B7803B908BDFFF7EAFF0028FAD065
:1076F0000720FFF7D9FFF6E7641E002008B5FFF763
:10770000DFFF18B10D20FFF7CFFF08BD0C20FFF7FA
:10771000CBFFFAE720B1034B9A89024B5A607047BE
:107720000022FAE7641E002008B5034B187000B170
:1077300008BDFFF7B1FFFBE7641E0020014B18787E
:10774000704700BF641E002010B44308332822D9BC
:10775000C3F132031E4A02EBC30052F833204468DF
:107760001C4BA3FB01031B09322000FB1313DBB2EC
:10777000C3F12000A3F1200122FA03F304FA00F080
:10778000034324FA01F10B4313F0010F0CBF012056
:10779000002010BC70470E4A02EBC30452F83300BD
:1077A00064680C4BA3FB01231B09322202FB13115B
:1077B000C9B2C1F12002A1F12003C84004FA02F2CB
:1077C000104324FA03F3184300F00100E1E700BF7F
:1077D000389600081F85EB5108B50023202B11DCDB
:1077E000028840F6FF718A420CD081888A4202D812
:1077F00004300133F2E70C4A92F8B4116FF34101FF
:1078000082F8B411212B00D008BD074B93F8B421A6
:107810006FF3410283F8B42103460722C2210348D3
:10782000FBF735F8F0E700BF20040020EFBEADDE27
:1078300010B5144C94F8B43143F0020384F8B43119
:107840001148FFF7C9FF1148FFF7C6FF1048FFF7BF
:10785000C3FF1048FFF7C0FF0F48FFF7BDFF0F48F9
:10786000FFF7BAFF0E48FFF7B7FF94F8B43113F0F3
:10787000020F00D010BD0322C3210A48FBF716F8FF
:10788000F8E700BF2004002050940008BC940008D2
:10789000009500084895000898950008F0950008A4
:1078A00000960008EFBEADDE0346064A126822B11C
:1078B000044A1068034413607047024A0249116089
:1078C000F6E700BF781E002000400020234A13681E
:1078D0000133136013F0020118D0214A4FF48010D5
:1078E00010614FF4002010611E4A12689289F2B1B3
:1078F0001B4A202010611C4A526A12F0010F1BD152
:1079000039B31A4B4FF400421A617047164AB2F964
:10791000BC21002A02DD124A10201061124AB2F97D
:10792000BE21002AE0DD0E4A08201061DCE70C4A87
:107930004FF400101061DEE713F0040F04D00B4B7E
:107940004FF400421A617047084B4FF000421A6131
:107950007047064B4FF000421A6170477C1E0020B2
:10796000000C01401C0300202004002000080140FE
:1079700008B5FBF7BDFE2F4A938F0133938792F82A
:1079800038300133DBB282F83830042B06D0294A74
:107990001364294A52F82330984708BD002382F81F
:1079A000383092F839300133DBB282F839300A2BA3
:1079B00009D003EB83014A001E490A641F4A52F8AA
:1079C00023309847E9E7002382F8393092F83A30BB
:1079D0000133DBB282F83A300A2B09D0642203FB70
:1079E00002F214490A64164A52F823309847D4E741
:1079F000002382F83A3092F83B300133DBB282F850
:107A00003B300A2B0CD00B4991F83B204FF47A7392
:107A100002FB03F30B640B4B53F822309847BCE78F
:107A20001346002182F83B10926A01329A629987CC
:107A3000E9E700BF2004002080970008589700085D
:107A40003097000808970008002300E001338342C4
:107A5000FCD3704770B54FF0FF0C4CF4E06C1CEA9F
:107A600011541DBF1CEA135594EA0C0F95EA0C0F34
:107A700000F0DEF82C4481EA030621EA4C5123EAA7
:107A80004C5350EA013518BF52EA033541F48011D6
:107A900043F4801338D0A0FB02CE4FF00005E1FB89
:107AA00002E506F00042E0FB03E54FF00006E1FBD3
:107AB00003569CF0000F18BF4EF0010EA4F1FF0416
:107AC000B6F5007F64F5407404D25FEA4E0E6D4156
:107AD00046EB060642EAC62141EA55514FEAC52067
:107AE00040EA5E504FEACE2EB4F1FD0C88BFBCF5E3
:107AF000E06F1ED8BEF1004F08BF5FEA500E50F194
:107B0000000041EB045170BD06F0004646EA010159
:107B100040EA020081EA0301B4EB5C04C2BFD4EB8B
:107B20000C0541EA045170BD41F480114FF0000E84
:107B3000013C00F3AB8014F1360FDEBF002001F0F2
:107B4000004170BDC4F10004203C35DA0C341BDC6C
:107B500004F11404C4F1200500FA05F320FA04F03E
:107B600001FA05F240EA020001F0004221F0004172
:107B700010EBD37021FA04F642EB06015EEA430EE5
:107B800008BF20EAD37070BDC4F10C04C4F1200515
:107B900000FA04F320FA05F001FA04F240EA0200C8
:107BA00001F0004110EBD37041F100015EEA430E99
:107BB00008BF20EAD37070BDC4F1200500FA05F2B9
:107BC0004EEA020E20FA04F301FA05F243EA020338
:107BD00021FA04F001F0004121FA04F220EA020047
:107BE00000EBD3705EEA430E08BF20EAD37070BD8D
:107BF00094F0000F0FD101F00046400041EB01016D
:107C000011F4801F08BF013CF7D041EA060195F04E
:107C1000000F18BF704703F00046520043EB030308
:107C200013F4801F08BF013DF7D043EA06037047F5
:107C300094EA0C0F0CEA135518BF95EA0C0F0CD000
:107C400050EA410618BF52EA4306D1D181EA030146
:107C500001F000414FF0000070BD50EA410606BF40
:107C60001046194652EA430619D094EA0C0F02D185
:107C700050EA013613D195EA0C0F05D152EA0336CA
:107C80001CBF104619460AD181EA030101F00041E8
:107C900041F0FE4141F470014FF0000070BD41F031
:107CA000FE4141F4780170BD81F0004102E000BF67
:107CB00083F0004330B54FEA41044FEA430594EAAC
:107CC000050F08BF90EA020F1FBF54EA000C55EAE7
:107CD000020C7FEA645C7FEA655C00F0E2804FEAB8
:107CE0005454D4EB5555B8BF6D420CDD2C4480EA9A
:107CF000020281EA030382EA000083EA010180EACA
:107D0000020281EA0303362D88BF30BD11F0004F17
:107D10004FEA01314FF4801C4CEA113102D040424D
:107D200061EB410113F0004F4FEA03334CEA133388
:107D300002D0524263EB430394EA050F00F0A780A0
:107D4000A4F10104D5F1200E0DDB02FA0EFC22FA9B
:107D500005F2801841F1000103FA0EF2801843FA8F
:107D600005F359410EE0A5F120050EF1200E012A80
:107D700003FA0EFC28BF4CF0020C43FA05F3C018BE
:107D800051EBE37101F0004507D54FF0000EDCF137
:107D9000000C7EEB00006EEB0101B1F5801F1BD3E0
:107DA000B1F5001F0CD349085FEA30004FEA3C0CE4
:107DB00004F101044FEA445212F5800F80F09A80DA
:107DC000BCF1004F08BF5FEA500C50F1000041EBDE
:107DD000045141EA050130BD5FEA4C0C404141EBE2
:107DE0000101013C28BFB1F5801FE9D291F0000FDD
:107DF00004BF01460020B1FA81F308BF2033A3F18C
:107E00000B03B3F120020CDA0C3208DD02F1140C82
:107E1000C2F10C0201FA0CF021FA02F10CE002F1BD
:107E20001402D8BFC2F1200C01FA02F120FA0CFCB6
:107E3000DCBF41EA0C019040E41AA2BF01EB0451FF
:107E4000294330BD6FEA04041F3C1CDA0C340EDCFD
:107E500004F11404C4F1200220FA04F001FA02F340
:107E600040EA030021FA04F345EA030130BDC4F1FE
:107E70000C04C4F1200220FA02F001FA04F340EAF3
:107E80000300294630BD21FA04F0294630BD94F0A4
:107E9000000F83F4801306BF81F480110134013D8B
:107EA0004EE77FEA645C18BF7FEA655C29D094EAFC
:107EB000050F08BF90EA020F05D054EA000C04BF7A
:107EC0001946104630BD91EA030F1EBF0021002065
:107ED00030BD5FEA545C05D14000494128BF41F004
:107EE000004130BD14F580043CBF01F5801130BD68
:107EF00001F0004545F0FE4141F470014FF00000F3
:107F000030BD7FEA645C1ABF194610467FEA655CA3
:107F10001CBF0B46024650EA013406BF52EA033545
:107F200091EA030F41F4002130BD00BF90F0000F33
:107F300004BF0021704730B54FF4806404F132046F
:107F40004FF000054FF0000150E700BF90F0000F28
:107F500004BF0021704730B54FF4806404F132044F
:107F600010F0004548BF40424FF000013EE700BF1F
:107F700042004FEAE2014FEA31014FEA02701FBFAF
:107F800012F07F4393F07F4F81F06051704732F0E1
:107F90007F4208BF704793F07F4F04BF41F4002138
:107FA000704730B54FF4607401F0004521F0004196
:107FB0001CE700BF50EA010208BF704730B54FF020
:107FC00000050AE050EA010208BF704730B511F021
:107FD000004502D5404261EB41014FF4806404F159
:107FE00032045FEA915C3FF4D8AE4FF003025FEADF
:107FF000DC0C18BF03325FEADC0C18BF033202EB63
:10800000DC02C2F1200300FA03FC20FA02F001FABC
:1080100003FE40EA0E0021FA02F11444BDE600BF5F
:108020004FF0FF3C06E000BF4FF0010C02E000BF44
:108030004FF0010C4DF804CD4FEA410C7FEA6C5C27
:108040004FEA430C18BF7FEA6C5C1BD001B050EACA
:10805000410C0CBF52EA430C91EA030F02BF90EAB5
:10806000020F0020704710F1000F91EA030F58BF74
:10807000994208BF90422CBFD8176FEAE37040F0D6
:10808000010070474FEA410C7FEA6C5C02D150EA74
:10809000013C07D14FEA430C7FEA6C5CD6D152EA2F
:1080A000033CD3D05DF8040B704700BF84461046F4
:1080B00062468C461946634600E000BF01B5FFF7F3
:1080C000B7FF002848BF10F1000F01BD4DF808EDC3
:1080D000FFF7F4FF0CBF012000205DF808FB00BF94
:1080E0004DF808EDFFF7EAFF34BF012000205DF8EE
:1080F00008FB00BF4DF808EDFFF7E0FF94BF01203B
:1081000000205DF808FB00BF4DF808EDFFF7CEFF3B
:1081100094BF012000205DF808FB00BF4DF808ED7A
:10812000FFF7C4FF34BF012000205DF808FB00BF4B
:108130004FEA4102B2F1E04324BFB3F5001CDCF189
:10814000FE5C0DD901F0004C4FEAC0024CEA5070C1
:10815000B2F1004F40EB830008BF20F001007047F0
:1081600011F0804F21D113F13872BCBF01F00040F3
:10817000704741F480114FEA5252C2F11802C2F125
:10818000200C10FA0CF320FA02F018BF40F00100A6
:108190004FEAC1234FEAD32303FA0CFC40EA0C0058
:1081A00023FA02F34FEA4303CCE77FEA625307D195
:1081B00050EA01331EBF4FF0FE4040F440007047CC
:1081C00001F0004040F0FE4040F40000704700BF66
:1081D00080F0004002E000BF81F0004142001FBF7C
:1081E0005FEA410392EA030F7FEA226C7FEA236C85
:1081F0006AD04FEA1262D2EB1363C1BFD21841407A
:1082000048404140B8BF5B42192B88BF704710F00F
:10821000004F40F4000020F07F4018BF404211F0B2
:10822000004F41F4000121F07F4118BF494292EA1A
:10823000030F3FD0A2F1010241FA03FC10EB0C0046
:10824000C3F1200301FA03F100F0004302D54942D3
:1082500060EB4000B0F5000F13D3B0F1807F06D380
:1082600040084FEA310102F10102FE2A51D2B1F178
:10827000004F40EBC25008BF20F0010040EA03006D
:108280007047490040EB0000013A28BFB0F5000FED
:10829000EDD2B0FA80FCACF1080CB2EB0C0200FAA3
:1082A0000CF0AABF00EBC25052421843BCBFD040F2
:1082B0001843704792F0000F81F4000106BF80F46C
:1082C00000000132013BB5E74FEA41037FEA226C2F
:1082D00018BF7FEA236C21D092EA030F04D092F0FA
:1082E000000F08BF0846704790EA010F1CBF00202E
:1082F000704712F07F4F04D1400028BF40F000408B
:10830000704712F100723CBF00F50000704700F0AA
:10831000004343F0FE4040F4000070477FEA2262D1
:1083200016BF08467FEA23630146420206BF5FEAA2
:10833000412390EA010F40F4800070474FF00003A2
:1083400004E000BF10F0004348BF40425FEA000C69
:1083500008BF704743F0964301464FF000001CE011
:1083600050EA010208BF70474FF000030AE000BF67
:1083700050EA010208BF704711F0004302D54042A5
:1083800061EB41015FEA010C02BF84460146002017
:1083900043F0B64308BFA3F18053A3F50003BCFA32
:1083A0008CF2083AA3EBC25310DB01FA02FC6344DF
:1083B00000FA02FCC2F12002BCF1004F20FA02F2E6
:1083C00043EB020008BF20F00100704702F12002D9
:1083D00001FA02FCC2F1200250EA4C0021FA02F23A
:1083E00043EB020008BF20EADC7070474FF0FF0C3F
:1083F0001CEAD0521EBF1CEAD15392EA0C0F93EA3A
:108400000C0F6FD01A4480EA010C400218BF5FEADB
:1084100041211ED04FF0006343EA501043EA51114E
:10842000A0FB01310CF00040B1F5000F3EBF490048
:1084300041EAD3715B0040EA010062F17F02FD2A4C
:108440001DD8B3F1004F40EBC25008BF20F001002F
:10845000704790F0000F0CF0004C08BF49024CEA46
:10846000502040EA51207F3AC2BFD2F1FF0340EAD8
:10847000C250704740F400004FF00003013A5DDC49
:1084800012F1190FDCBF00F000407047C2F100028A
:10849000410021FA02F1C2F1200200FA02FC5FEA77
:1084A000310040F1000053EA4C0308BF20EADC70C1
:1084B000704792F0000F00F0004C02BF400010F433
:1084C000000F013AF9D040EA0C0093F0000F01F0E0
:1084D000004C02BF490011F4000F013BF9D041EA02
:1084E0000C018FE70CEAD15392EA0C0F18BF93EA04
:1084F0000C0F0AD030F0004C18BF31F0004CD8D12E
:1085000080EA010000F00040704790F0000F17BFB4
:1085100090F0004F084691F0000F91F0004F14D0FA
:1085200092EA0C0F01D142020FD193EA0C0F03D152
:108530004B0218BF084608D180EA010000F0004055
:1085400040F0FE4040F40000704740F0FE4040F430
:10855000400070474FF0FF0C1CEAD0521EBF1CEACF
:10856000D15392EA0C0F93EA0C0F69D0A2EB0302ED
:1085700080EA010C49024FEA402037D04FF0805387
:1085800043EA111143EA10130CF000408B4238BF4C
:108590005B0042F17D024FF4000C8B4224BF5B1A5A
:1085A00040EA0C00B3EB510F24BFA3EB510340EAA8
:1085B0005C00B3EB910F24BFA3EB910340EA9C0056
:1085C000B3EBD10F24BFA3EBD10340EADC001B01C6
:1085D00018BF5FEA1C1CE0D1FD2A3FF650AF8B426A
:1085E00040EBC25008BF20F0010070470CF0004C77
:1085F0004CEA50207F32C2BFD2F1FF0340EAC250A2
:10860000704740F400004FF00003013A37E792F062
:10861000000F00F0004C02BF400010F4000F013AC0
:10862000F9D040EA0C0093F0000F01F0004C02BFBB
:10863000490011F4000F013BF9D041EA0C0195E724
:108640000CEAD15392EA0C0F08D142027FF47DAFBD
:1086500093EA0C0F7FF470AF084676E793EA0C0FAD
:1086600004D14B023FF44CAF08466EE730F0004CAB
:1086700018BF31F0004CCAD130F000427FF45CAF3B
:1086800031F000437FF43CAF5FE700BF4FF0FF3CA9
:1086900006E000BF4FF0010C02E000BF4FF0010CFC
:1086A0004DF804CD4FEA40024FEA41037FEA226CC5
:1086B00018BF7FEA236C11D001B052EA530C18BFE7
:1086C00090EA010F58BFB2EB030088BFC81738BF4C
:1086D0006FEAE17018BF40F0010070477FEA226C3A
:1086E00002D15FEA402C05D17FEA236CE4D15FEA36
:1086F000412CE1D05DF8040B704700BF844608466A
:108700006146FFE70FB5FFF7C9FF002848BF10F12A
:10871000000F0FBD4DF808EDFFF7F4FF0CBF01206F
:1087200000205DF808FB00BF4DF808EDFFF7EAFFF9
:1087300034BF012000205DF808FB00BF4DF808EDB4
:10874000FFF7E0FF94BF012000205DF808FB00BFA9
:108750004DF808EDFFF7D2FF94BF012000205DF82F
:1087600008FB00BF4DF808EDFFF7C8FF34BF01203C
:1087700000205DF808FB00BF4FEA4002B2F1FE4F57
:108780000FD34FF09E03B3EB12620DD94FEA0023D3
:1087900043F0004310F0004F23FA02F018BF4042AC
:1087A00070474FF00000704712F1610F01D1420293
:1087B00005D110F0004008BF6FF0004070474FF047
:1087C0000000704742000ED2B2F1FE4F0BD34FF0C3
:1087D0009E03B3EB126209D44FEA002343F0004337
:1087E00023FA02F070474FF00000704712F1610F5A
:1087F00001D1420202D14FF0FF3070474FF000002C
:10880000704700BF0EB46FF0004100B59CB01DABC7
:1088100002900690079104910848094953F8042BE7
:108820000591006802A9019300F07EF90022029BE5
:108830001A701CB05DF804EB03B0704734030020DD
:108840000802FFFF03460244934200D1704703F839
:10885000011BF9E7704770470A44914200F1FF336A
:1088600000D1704710B511F8014B914203F8014F48
:10887000F9D110BD034613F8012B002AFBD1181AB9
:108880000138704738B50546002940D051F8043CFE
:108890000C1F002BB8BFE41800F0DEF81C4A136868
:1088A00033B9636014602846BDE8384000F0DAB898
:1088B000A34208D9206821188B4201BF19685B6860
:1088C00009182160EDE71A465B680BB1A342FAD99B
:1088D00011685018A0420BD12068014450188342FF
:1088E0001160E0D118685B68084410605360DAE7F3
:1088F00002D90C232B60D6E7206821188B4201BFD8
:1089000019685B680918216063605460CBE738BD63
:10891000C41F002070B50F4E0C463168054611B9D2
:1089200000F0B6FB30602146284600F0B1FB431C46
:1089300003D14FF0FF34204670BDC41C24F0030463
:10894000A042F8D0211A284600F0A2FB0130F2D153
:10895000EFE700BFC01F00202DE9F843CD1C25F034
:10896000030508350C2D38BF0C25002D064601DB0C
:10897000A94204D90C2333600020BDE8F883DFF856
:10898000D48000F069F8D8F800301C4644BB294672
:108990003046FFF7BFFF431C044658D1D8F80040CB
:1089A0002746002F43D1002C4BD023683946304650
:1089B00004EB030900F06CFB814542D1216830468D
:1089C0006D1A2946FFF7A6FF01303AD023682B44E1
:1089D0002360D8F800305A6862BBC8F800700FE016
:1089E0002268521B20D40B2A17D96119A342256093
:1089F00018BF5960636808BFC8F8001062514B6027
:108A0000304600F02FF804F10B00231D20F0070082
:108A1000C21A1CBF1B1AA350AFE76268A3420CBF67
:108A2000C8F800205A60EBE723466468AEE73C468E
:108A30007F68B6E71A465B68A342FBD10023536008
:108A4000DEE70C233046336000F00CF894E7056055
:108A5000D6E700BFC41F00200148FFF7FBBE00BFE0
:108A6000BC1F00200148FFF7F6BE00BFBC1F00205E
:108A70002DE9F0471F468E688246BE420C4690465E
:108A80000B682DD8B1F90C2012F4906F26D06569CF
:108A9000096905EB4505A3EB010905EBD5757B1CC1
:108AA0004B446D109D4238BF1D46530527D52946BE
:108AB000FFF752FF064660B34A462169FFF7CCFE36
:108AC000A38923F4906343F08003A38126614E447D
:108AD00026603E466561A5EB0905A560BE4200D94A
:108AE0003E4632464146206800F0B8FA0020A368AE
:108AF0009B1BA360236833442360BDE8F0872A46AC
:108B000000F0E4FA06460028E0D150462169FFF75C
:108B1000B9FE0C23CAF80030A3894FF0FF3043F0B0
:108B20004003A381E9E700002DE9F04F98468B89C7
:108B300007461B060D4614469DB010D50B6973B948
:108B40004021FFF709FF2860286130B90C233B6002
:108B50004FF0FF301DB0BDE8F08F40236B61002364
:108B6000099320238DF8293030234FF00109CDF8E7
:108B70000C80DFF898818DF82A3023469A4613F846
:108B8000012B0AB1252AF9D1BAEB040B0BD05B46B5
:108B9000224629463846FFF76BFF013000F0A780D8
:108BA000099A5A4409929AF80030002B00F09F80ED
:108BB00000234FF0FF32CDE905230AF1010A0493A7
:108BC00007938DF853301A935446052214F8011B6D
:108BD0004E4800F06DFA049AD8B9D00644BF20235D
:108BE0008DF85330110744BF2B238DF853309AF87A
:108BF00000302A2B15D0544600204FF00A0C079A5B
:108C0000214611F8013B303B092B4BD9B0B10792FB
:108C100014E0A0EB080309FA03F31343A2460493FC
:108C2000D2E7039B191D1B680391002BBBBF5B425E
:108C300042F0020207930793B8BF049223782E2BC9
:108C40000AD163782A2B32D1039B02341A1D1B6888
:108C5000039243EAE3730593DFF8B4A0032250467E
:108C6000217800F025FA38B14022049BA0EB0A00DD
:108C7000824013430134049314F8011B0622254853
:108C80008DF8281000F014FA002836D0224B1BBBB8
:108C9000039B073323F0070308330393099B3344F3
:108CA00009936AE70C4601200CFB0232A8E7002377
:108CB0004FF00A0C194601340593204610F8012B99
:108CC000303A092A03D9002BC6D00591C4E70446DF
:108CD00001230CFB0121F0E703AB00932A46384641
:108CE0000E4B04A9AFF30080421C0646D6D1AB89D7
:108CF0005B063FF52DAF09982CE703AB00932A469E
:108D00003846064B04A900F07DF8EDE7909700087F
:108D1000969700089A97000800000000718A0008E2
:108D20002DE9F047164698468A680B690746934234
:108D3000B8BF1346336091F843200C46DDF820900D
:108D40000AB1013333602368990642BF33680233A6
:108D50003360256815F0060506D104F1190AE368A9
:108D600032689B1AAB422BDC94F843302268003BFC
:108D700018BF0123920630D44146384604F143021D
:108D8000C847013023D02368226903F00603042B6F
:108D900014BF002533684FF0000608BFE56804F1F2
:108DA0001A0408BFED1A54F8123C08BF25EAE5750D
:108DB0009342C4BF9B1AED18B5421AD1002008E0B7
:108DC0000123524641463846C847013003D14FF08F
:108DD000FF30BDE8F0870135C1E73020E11881F8A8
:108DE00043005A1C94F845102244023382F8431081
:108DF000C2E70123224641463846C8470130E6D043
:108E00000136D9E72DE9FF470F7E9146782F80463E
:108E10000C469A460C9E01F1430207D8622F0AD8ED
:108E2000002F00F0DD80582F00F0C38004F14206CF
:108E300084F842703AE0A7F16303152BF6D801A13C
:108E400051F823F09D8E0008B18E00082D8E000889
:108E50002D8E00082D8E00082D8E0008B18E000882
:108E60002D8E00082D8E00082D8E00082D8E0008F6
:108E7000C78F00083F8F00087F8F00082D8E0008E5
:108E80002D8E0008E98F00082D8E00083F8F000806
:108E90002D8E00082D8E0008878F000833681A1D5C
:108EA0001B68326004F1420684F842300123A8E0D6
:108EB00031682368081D30601E0601D50D6803E087
:108EC0005D06FBD5B1F90050002D616878DA2D20E0
:108ED000002984F84300A1602DDA0A235D486D4221
:108EE0001646B5FBF3F103FB1157C75D06F8017D8C
:108EF0002F46BB420D46F4D9082B0BD12368DF0760
:108F000008D5236961689942DEBF302306F8013C29
:108F100006F1FF36921B22614B4621464046CDF8B2
:108F200000A003AAFFF7FCFE01306FD14FF0FF3025
:108F300004B0BDE8F08723F004032360CDE7216887
:108F40003368080653F8045B02D4490648BFADB243
:108F50006F2F336014BF0A2308233E48002184F892
:108F600043106668002EA660BADB216821F0040178
:108F70002160002DB4D1002EB2D11646BCE7236883
:108F800043F0200323607827334884F84570236832
:108F900031681F0651F8045B02D45F0648BFADB2CA
:108FA0003160D90744BF43F0200323601DB1102373
:108FB000D4E72848E9E7236823F020032360F6E795
:108FC0000A232448CDE733682568181D616930609D
:108FD0002E061B6801D5196002E06806FBD51980D2
:108FE00000231646236197E7336800211A1D32607B
:108FF0001E686268304600F05BF808B1801B606054
:1090000063682361002384F8433085E7324649468C
:1090100040462369D047013088D023689B0714D489
:10902000E068039B9842B8BF184681E701233246A7
:1090300049464046D04701303FF478AF0135E368F8
:1090400003995B1AAB42F1DCEAE7002504F119064B
:10905000F5E700BFA1970008B2970008884210B555
:1090600001EB020402D98442234607D8431EA142E1
:1090700008D011F8012B03F8012FF8E7014602444C
:109080008A4200D110BD13F8014D02F8014DF7E7F7
:1090900038B50023054D044608462B60FEF704FC56
:1090A000431C02D12B6803B1236038BDB81F0020D8
:1090B000034610B5C9B202449342184601D10020BC
:1090C00003E0047801338C42F6D110BD2DE9F04164
:1090D000804615460C4621B91146BDE8F041FFF720
:1090E0003BBC2AB9FFF7CEFB00242046BDE8F08147
:1090F00000F01AF88542064602D8B5EB500FF4D8B6
:1091000029464046FFF728FC07460028ECD0B54228
:109110002A46214628BF3246FFF79EFB214640469D
:10912000FFF7B0FB3C46E0E751F8043C181F002B6A
:10913000BCBF0B58C0187047F8B500BFF8BC08BCDE
:109140009E467047F8B500BFF8BC08BC9E46704705
:10915000256420002535642000000000307825308B
:10916000327820003078253034782000307825306F
:10917000387820002573200025642E2530336400C4
:10918000253032582000000046616C7365000000F5
:109190005472756500000000545420320000000035
:1091A0004842202020202020000000002D2D2D2DC1
:1091B0002D2D2D2D00000000545420310000000002
:1091C0005041305F52544432000000005041315F42
:1091D00052544431000000005041335F495345541C
:1091E000000000005041345F52544433000000003E
:1091F00042315F43414E4144440000004348505FC8
:10920000544D50002544555459000000564F4C54BD
:109210005300000043616E204144445200000000AE
:1092200054656D700000000077617468646F6700BA
:109230004B4D3A56352E30303700000054454D50D6
:10924000630000004B4661637400000044545F42B9
:109250004941530046414E5F4D5800004F767254CD
:109260006D700000000000000000005F00000007BB
:10927000000700147F147F14242A7F2A1223130866
:10928000646236495522500005030000001C22414B
:10929000000041221C00082A1C2A0808083E080871
:1092A0000050300000080808080800606000002036
:1092B000100804023E5149453E00427F4000426191
:1092C0005149462141454B311814127F102745451D
:1092D00045393C4A49493001710905033649494934
:1092E00036064949291E0036360000005636000071
:1092F000000814224114141414144122140800020A
:1093000001510906324979413E7E1111117E7F4992
:109310004949363E414141227F4141221C7F494912
:1093200049417F090901013E414151327F08080846
:109330007F00417F41002040413F017F08142241CE
:109340007F404040407F0204027F7F0408107F3E40
:109350004141413E7F090909063E4151215E7F0995
:10936000192946464949493101017F01013F4040E1
:10937000403F1F2040201F7F2018207F63140814C7
:10938000630304780403615149454300007F414170
:10939000020408102041417F000004020102044041
:1093A00040404040000102040020545454787F485B
:1093B0004444383844444420384444487F38545462
:1093C0005418087E090102081454543C7F08040410
:1093D0007800447D40002040443D00007F10284438
:1093E00000417F40007C041804787C08040478382D
:1093F000444444387C14141408081414187C7C0861
:109400000404084854545420043F4440203C404045
:10941000207C1C2040201C3C4030403C442810282C
:10942000440C5050503C4464544C440008364100B5
:1094300000007F0000004136080008082A1C0808C8
:109440001C2A0808553500008A0D55350122AD0D3E
:109450006C005B0026011A00C40110007B0215009D
:1094600024030B00AF0316003A040C00CC041700D1
:109470006D050D001B061800D7060E009A0719008F
:109480005C080F0029095C00F0092E00A30A2400E3
:10949000550B2900F90B1F00800C2A00F50C200049
:1094A0006F0D2B00E50D2100530E2C00C40E220081
:1094B000420F2D00C20F2300FF0FFE000000603599
:1094C0002A00E021550260109B02C00F4103800E6C
:1094D0000F04400D0805000C2C06C00A790780090E
:1094E000DE084008490A0007A10BC005D10C800422
:1094F000CA0D4003890E0002080FE000FF0F0000B4
:109500000000603590018020F401401F1C02E01E25
:109510007602001EE902C01C9603401BEB03A01A52
:10952000DA0420194D062017C6090013240C201058
:10953000DE0D400D3C0FE008860FC006B00F200482
:10954000F00F6000FF0F00000000C0E15B0100E7CA
:10955000A60240EDB40380F39504C0F95505000060
:10956000FB0540068C06800C0B07C0127C07001917
:10957000E107401F3B0880258D08C02BD70800322B
:109580001A0940385809803E9009C044C409004B6C
:10959000F90AE07CFF0F2C01000000198E02401038
:1095A0002103000FD303C00DA804800CA305400BBA
:1095B000C106000AFC07C00847098007910A400657
:1095C000C80B0005DC0CC003550D2003C10D800243
:1095D000750E4001FC0E00005B0FC0FE9B0F80FD6E
:1095E000C40F40FCDE0F00FBED0FC0F9FF0F018040
:1095F00000000000F4018200E8030401FF0F57049B
:10960000000080DF9F00C0F9C3000000D10080028D
:10961000DF000005ED008007FB00000A0901800C57
:109620002B01C0124D0100196E01401F0A02803E3D
:109630001F03E07CFF0F2C01000000000000000071
:109640000100000000000000010000020000000016
:1096500001000200040000000120000240000000A0
:109660000104104000010000010202020404000095
:1096700001814020100800008120080241100000F4
:10968000410842108210000021841042082100008D
:109690002142840811220000212222424444000079
:1096A0001111118988880000118944221289000053
:1096B00091441249249100009124492249920000CA
:1096C0004992244992240100494A529292940000FE
:1096D000494949292929010029A594524A2901000B
:1096E000A9542A954AA5000055952A55A95201006A
:1096F000A92A55A5AA540100555555AAAAAA0000A1
:109700005555555555550100EF2800087929000891
:10971000EF280008EF280008EF280008EF280008CD
:10972000EF280008EF280008EF2800085538000847
:10973000F12800082D3400085D2900088D39000843
:10974000EF280008EF280008B52F0008CD780008A2
:10975000EF28000829290008F1280008EF28000850
:10976000EF280008B1410008454D0008EF28000827
:10977000DD44000815390008DD49000825290008E6
:10978000F12800083D520008371700084946000834
:10979000232D302B2000686C4C00656667454647DA
:1097A000003031323334353637383941424344455D
:1097B00046003031323334353637383961626364CC
:0397C000656600DB
:0897C400B0F0FF7F010000007E
:1097CC0000A24A040204060800000000010203047F
:1097DC000102030406070809AC0300200100000085
:1097EC0098910008000000F81FF80000000000002D
:1097FC004E0202007C1E0020A09100080100FFFF19
:10980C001FF80000000000004E16020000000000CF
:10981C00AC9100080100FFFF1FF8000000000000E1
:10982C004E2A020001000000B8910008000000F868
:10983C001FF80000000000004E0202007C1E0020F9
:10984C00A09100080100FFFF1FF8000000000000BD
:10985C004E160200D41D0020C09100080200FFFF2C
:10986C001FF800000000000044320100D61D00204B
:10987C00CC9100080200FFFF1FF800000000000060
:10988C00443C0100D81D0020D89100080200FFFFC5
:10989C001FF800000000000044460100DA1D002003
:1098AC00E49100080200FFFF1FF800000000000018
:1098BC0044500100DC1D0020F09100080200FFFF65
:1098CC001FF8000000000000445A0100DE1D0020BB
:1098DC00FC9100080200FFFF1FF8000000000000D0
:1098EC004464010000000000AC9100080100FFFF7F
:1098FC001FF8000000000000447801001C04002048
:10990C00049200080200FFFF1FF800000000000096
:10991C00440A02001C040020A89100080A001FF849
:10992C000000000000000000001E0200CC1D002002
:10993C00A89100080000FFFF1FF8000000000000C5
:10994C0000320100CC1D00200C9200080300FFFF28
:10995C001FF8000000000000443C0100C41D002062
:10996C00149200080200FFFF1FF800000000000026
:10997C0044460100C81D0020DC9100080300FFFFD5
:10998C001FF800000000000044500100D01D002012
:10999C00209200080300FFFF1FF8000000000000E9
:1099AC00445A0100661A0020289200080200FFFFAA
:1099BC001FF8000000000000446401007C1E002021
:1099CC0030920008010000F81FF8000000000000B1
:1099DC00446E010000000000AC9100080100FFFF84
:1099EC001FF800000000000044780100CC050020A6
:1099FC003C9200080300FFFF1FF80000000000006D
:109A0C004405020090050020049200080200FFFFAC
:109A1C001FF8000000000000441E0200CC1D0020B6
:109A2C00A89100080000FFFF1FF8000000000000D4
:109A3C0000320100D0050020449200080300FFFF13
:109A4C001FF8000000000000443C0100240300202B
:109A5C004C9200080300FFFF1FF8000000000000FC
:109A6C0044460100B4050020549200080200FFFF98
:109A7C001FF800000000000044500100B005002059
:109A8C005C9200080200FFFF1FF8000000000000BD
:109A9C00445A0100661A0020289200080200FFFFB9
:109AAC001FF8000000000000446401007C1E002030
:109ABC0030920008010000F81FF8000000000000C0
:109ACC00446E010000000000AC9100080100FFFF93
:109ADC001FF800000000000044780100340500204D
:109AEC00840500200000803F0A00000038328F3BC4
:109AFC0017B7513A3803002000000000801E0020E8
:109B0C00E81E0020501F0020000000000000000094
:109B1C000000000000000000000000000000000039
:109B2C000000000000000000000000000000000029
:109B3C000000000000000000000000000000000019
:0C9B4C0000000000750100084D01000839
:0400000508000000EF
:00000001FF
